:10D7FA00202020002D2D2D002533730025336400B1
:10D80A00452530326400502531642E25316400509C
:10D81A00253032640025342E316600432531642ECA
:10D82A0025316400432530326400253031642E25C9
:04D83A003032640024
:10B51800C211E4FFEF25E025E02426F582E4340299
:10B52800F5837407F0EF25E025E02428F582E4345C
:10B5380002F583E4F0741B2FF582E43402F583E40A
:10B54800F00FEFB40ACEE4900239F090023B04F019
:10B55800E4900235F09002377402F0E4900231F082
:10B568009002337404F0E490022DF090022F7408D6
:10B57800F0E4900229F090022B7410F0E490022578
:10B58800F09002277420F09002497401F090024B69
:10B59800F090023DF090023F7408F090024174016F
:10B5A800F09002437404F09002457401F090024751
:10B5B80004F07B0190012914F0A37402F0A3741223
:10B5C800F09000EB74FFF0A374D7F0A374FAF07A4C
:10B5D800027912126C1390012C7401F0A37403F019
:10B5E800800690012D7404F0E490012EF0A3F0A3DE
:10B5F800F0A3F0A3F0A37402F07B0190017714F09C
:10B60800A37402F0A37417F09000EB74FFF0A37416
:10B61800D7F0A374FAF07A027917126C1390017AB2
:10B628007401F0A37403F0E4A3F0A3F0A3F0A3F073
:09B63800A3F0A37402F012CD800E
:01B6410022E6
:0BA7F7009000DFEBF0A3EAF0A3E9F014
:10A8020012303F78E47C007D011233267B017A000E
:10A8120079E412DE479000E3EFF078E47C007D01FA
:10A822007BFF7AD779FE12323DEF700302A91C7BBF
:10A83200017A0079E47D2E12DC8DEFF47002EEF4E1
:10A842006054E49000E2F09000DFE0FBA3E0FAA3A2
:10A85200E0F990000A122CE0FD9000E2E0C39D5066
:10A86200089000E2E004F080DE74E52FF9E43400A1
:10A87200FA7B01C00174E42FF9E43400A801FC7DE5
:10A8820001D0011233267B017A0079E412DE47906F
:10A8920000E3EFF08024E49000E2F09000DFE0FBC0
:10A8A200A3E0FAA3E0F990000A122CE0FF9000E284
:10A8B200E0C39F5005E004F080E19000E4E0642DE5
:10A8C20070589000DFE0FBA3E0FAA3E0F9900004E7
:10A8D200122CE0FF9000E3E0FEEFC39E503C90009C
:10A8E200E5E0FFB43105745FF08012EFB4320890F6
:10A8F20000E5743DF080069000E5742AF078E47C6F
:10A90200007D017B017A0079E51233267B017A0012
:10A9120079E412DE479000E3EFF0E49000E2F09079
:10A9220000E3E0FF9000E2E0FEC39F506274E42E79
:10A93200F582E43400F583E0FF12D1DDEF75F00912
:10A94200A42431F974AE35F0FA7BFFC003C002C013
:10A95200019000DFE0FBA3E0FAA3E0F99000081207
:10A962002CE0FF9000E2E02FFF9000DFE0A3E0A3E5
:10A97200E0900009122CE0FD9000EF7405F0D00188
:0FA98200D002D00312D63F9000E2E004F08090A4
:01A9910022A3
:0BD72200900008EBF0A3EAF0A3E9F090
:10D72D00E4A3F0900008E0FBA3E0FAA3E0F9900079
:10D73D0004122CE0FF90000BE0FEC39F501E9000E2
:10D74D0008122CE0FFEE2FFF900009122CE0FD7B5C
:0CD75D000512D9EF90000BE004F080C72B
:01D76900229D
:10D036009000D0EBF0A3EAF0A3E9F09000D0E0FB7B
:10D04600A3E0FAA3E0F912303FC002C0019000EB62
:10D0560074FFF0A374D8F0A37402F09000D3E0F943
:10D06600A3E0FAA3E09000EEC9F0A3EAF0A3E9F08A
:10D07600D001D002126C139000D0E0FBA3E0FAA31B
:10D08600E0F99000077401122D52900005E4122D6C
:0CD0960052900006E4122D5212A7F7225F
:10D8C0009000EB74FFF0A374D8F0A37406F0A3EEFD
:10D8D000F0A3EFF0900129E0FBA3E0FAA3E0F91236
:10D8E0006C1390012EE0701590013004F0E490016B
:0ED8F0002EF0A3F07B017A01792912A7F7220E
:10DEE300E490012EF0A3F07B017A01792912A7F7C0
:01DEF300220C
:10D8FE009000EB74FFF0A374D8F0A3740AF0A3E4C5
:10D90E00F0A3EFF07B017A027917126C1390017E6F
:10D91E007401F0E490017CF0A3F07B017A01797739
:0DD92E0012A7F77B017A01797712DAC02287
:10DA2800900184E0FEA3E0FF12D8C090019574FF36
:10DA3800F07F0112B642900173E0FEA3E0FF12B836
:10DA4800737F0912BEC6900121E0FEA3E0FF12C851
:07DA580005E4900195F022A6
:10C133009000D37401F0A37400F0A37406F0A37409
:10C1430001F0A37400F0A37407F0A37401F0A374C7
:10C1530000F0A37408F07B017A00790512C06690A1
:10C163000007E0603E9000EB74FFF0A374D8F0A3E7
:10C173007410F0900005E02401FEE4339000EEF02B
:10C18300A3CEF0900006E02401FEE4339000F0F02B
:10C19300A3CEF0900129E0FBA3E0FAA3E0F9126C2F
:10C1A30013802C9000EB74FFF0A374D8F0A37419E0
:10C1B300F0900005E02401FEE4339000EEF0A3CEFE
:10C1C300F0900129E0FBA3E0FAA3E0F9126C137BE2
:10C1D300017A007908127BE59001307401F0E49054
:0EC1E300012EF0A3F07B017A01792912A7F753
:01C1F100222B
:10C41D0090000B7401F0A37400F0A37407F07B017E
:10C42D007A00790512CC84900142E07002A3E0708D
:10C43D000590000704F012E0305071900007E0B451
:10C44D00012D9000EB74FFF0A374D8F0A37406F0E7
:10C45D00900005E0FFA3E09000EECFF0A3EFF09089
:10C46D000129E0FBA3E0FAA3E0F9126C13803D90E3
:10C47D000007E0B42136900005E0FCA3E0FDEC12CE
:10C48D002918E4FBFA792078401228769000EB7495
:10C49D00FFF0A374D8F0A3741FF0A3122FE2900144
:10C4AD0029E0FBA3E0FAA3E0F9126C1390013074BC
:10C4BD0001F0E490012EF0A3F07B017A01792912AD
:02C4CD00A7F7CF
:01C4CF00224A
:10D83E0012D68E7C007D0A122D869000EEEEF0A39D
:10D84E00EFF09000EB74FFF0A374D8F0A37406F021
:10D85E007B017A0079D0126C139000D77401F0A37B
:10D86E007400F0A374D0F07B017A01792912CA54A6
:01D87E002287
:10BD1C009000D67401F0A37400F0A37406F0A37421
:10BD2C0001F0A37400F0A37407F0A37401F0A374E2
:10BD3C0000F0A37409F0A37401F0A37400F0A374D1
:10BD4C0008F0A37401F0A37400F0A3740BF07B0152
:10BD5C007A00790512A992900007E0603E9000EB02
:10BD6C0074FFF0A374D8F0A37425F0900005E024C0
:10BD7C0001FEE4339000EEF0A3CEF0900006E02438
:10BD8C0001FEE4339000F0F0A3CEF0900129E0FB2B
:10BD9C00A3E0FAA3E0F9126C13802C9000EB74FF73
:10BDAC00F0A374D8F0A3742EF0900005E02401FEEB
:10BDBC00E4339000EEF0A3CEF0900129E0FBA3E079
:10BDCC00FAA3E0F9126C137B017A00790B127BE574
:10BDDC009001307401F0E490012EF0A3F07B017A15
:06BDEC0001792912A7F7FE
:01BDF200222E
:0592F500900005EFF000
:1092FA009000D67401F0A37400F0A37407F0A3746D
:10930A0001F0A37400F0A37408F0A37401F0A3742D
:10931A0000F0A3740AF0A37401F0A37400F0A3741C
:10932A0009F0A37401F0A37400F0A3740CF07B019C
:10933A007A00790612A992900009E0FF900005E0F0
:10934A0044E0FEEF5E900009F0900142E07002A353
:10935A00E0700590000904F0900008E0700302959F
:10936A0031A3E014605224FE70030294A624E27032
:10937A000302946D24E0700302942324C0606724DE
:10938A00FE70030294EA248160030295319000EB97
:10939A0074FFF0A374D8F0A37402F0A37401F0A3CD
:1093AA007400F0A3740CF0900129E0FBA3E0FAA387
:1093BA00E0F9126C130295319000EB74FFF0A3747C
:1093CA00D8F0A37406F090000AE0FFA3E09000EE44
:1093DA00CFF0A3EFF0900129E0FBA3E0FAA3E0F9B4
:1093EA00126C130295319000EB74FFF0A374D8F05D
:1093FA00A37406F090000BE02401FE90000AE0340A
:10940A00009000EEF0A3CEF0900129E0FBA3E0FA71
:10941A00A3E0F9126C130295319000EB74FFF0A3EC
:10942A0074D8F0A37434F090000AE0FAA3E0FB7C4D
:10943A00007D64FFAE02122D869000EEEEF0A3EFDF
:10944A00F07C007D64AF03AE02122D86A3ECF0A37C
:10945A00EDF0900129E0FBA3E0FAA3E0F9126C1306
:10946A0002953190000AE0FCA3E0FDEC122918E411
:10947A00FBFA792078401228769000EB74FFF0A36B
:10948A0074D8F0A3741FF0A3122FE2900129E0FB15
:10949A00A3E0FAA3E0F9126C130295319000EB7481
:1094AA00FFF0A374D8F0A37406F090000AE0FFA3BB
:1094BA00E09000EECFF0A3EFF0900129E0FBA3E0EB
:1094CA00FAA3E0F9126C139000D77401F0A37400A8
:1094DA00F0A3740CF07B017A01792912CA548047EF
:1094EA009000EB74FFF0A374D8F0A37406F0900018
:1094FA000BE02401FE90000AE034009000EEF0A395
:10950A00CEF0900129E0FBA3E0FAA3E0F9126C1374
:10951A009000D77401F0A37400F0A3740CF07B01DF
:10952A007A01792912CA549001307401F0E4900149
:0D953A002EF0A3F07B017A01792912A7F72A
:019547002201
:10DAC000900006122CE07023301109900007041218
:10DAD0002D528007900007E4122D5290000574FF2C
:0CDAE000122D5290000674FF122D5222ED
:10DD00009000077401122D52900005E4122D5290DC
:0ADD10000006E4122D5212A7F722BC
:10C9C200900005EBF0A3EAF0A3E9F0900005E0FB8C
:10C9D200A3E0FAA3E0F9900005122CE06073900046
:10C9E2000574FF122D0D900005122CE0603C9000A2
:10C9F20005E0FBA3E0FAA3E0F9900007122CE0FFA8
:10CA02006402604DEFB4010B900007E4122D521244
:10CA1200D72222900005E0FBA3E0FAA3E0F9900000
:10CA2200077401122D5212A7F722900005E0FBA312
:10CA3200E0FAA3E0F9900006122CE06009900005EC
:10CA420074FF122D52229000077401122D5212A768
:02CA5200F722C9
:0BCA54009000D4EBF0A3EAF0A3E9F09F
:10CA5F009000D4E0FBA3E0FAA3E0F912303F78DABC
:10CA6F007C007D011233269000D4E0FBA3E0FAA3F3
:10CA7F00E0F912303FA801AC02AD039000D7E0FB04
:10CA8F00A3E0FAA3E0F91233269000D4E0FBA3E071
:10CA9F00FAA3E0F912A7F79000D4E0FBA3E0FAA302
:10CAAF00E0F912303FA801AC02AD037B017A0079A7
:10CABF00DA1233269000D4E0FBA3E0FAA3E0F9905A
:10CACF0000077402122D529000057406122D529019
:06CADF000006E4122D52D6
:01CAE500222E
:10D2FA00E4FFFE122CC7FDEE25E025E02425F58289
:10D30A00E43402F583E06D703B900001122CE0FDDD
:10D31A00EE25E025E02426F582E43402F583E0B523
:10D32A000522EE25E025E02428F582E43402F5837F
:10D33A00E06011EE25E025E02427F582E43402F5C9
:09D34A0083E04FFF0EEEB40AAAC5
:01D3530022B7
:10D10D009000D2EFF0E0FF241BF582E43402F583AA
:10D11D00E0600312DF279000D2E0FE25E025E02439
:10D12D0028F582E43402F58374FFF0EE25E025E066
:10D13D002425F582E43402F583E0FCC004EE25E0FD
:10D14D0025E02426F582E43402F583E0FCEE75F04B
:10D15D0004A42425F9740235F0FA7B0112D2FAAB3E
:09D16D0007AD04D00712D87F229F
:10D54F00AE07EE25E025E02428F582E43402F583CA
:10D55F00E4F0EE25E025E02425F582E43402F5839E
:10D56F00E0FCC004EE25E025E02426F582E4340239
:10D57F00F583E0FCEF75F004A42425F9740235F06F
:10D58F00FA7B0112D2FAAB07AD04D00712D87F2273
:10CE7000AE07EE25E025E02428F582E43402F583B0
:10CE8000E06012EE25E025E02428F582E43402F586
:10CE900083E4F08011EE25E025E02428F582E434D7
:10CEA00002F58374FFF0EE25E025E02425F582E409
:10CEB0003402F583E0FCC004EE25E025E02426F5ED
:10CEC00082E43402F583E0FCAF06EF75F004A4249D
:10CED00025F9740235F0FA7B0112D2FAAB07AD04E2
:06CEE000D00712D87F22EA
:10CFC900B211E4900005F0900005E0FFC3940A5007
:10CFD9005B741B2FF582E43402F583E0B4FF0990FA
:10CFE9000005E012CE70803C900005E0FF241BF59F
:10CFF90082E43402F583E0602B900005E0FE241BF7
:10D00900F582E43402F583E014F0741B2EF582E412
:10D019003402F583E0600512CE708008900005E0C7
:0CD02900FF12D10D900005E004F0809B88
:01D0350022D8
:10DAEC009000D0EFF0A3EDF03011089000D0E0FFE3
:10DAFC0012D10D9000D1E0FF9000D0E0241BF582F4
:08DB0C00E43402F583EFF0227E
:10DF2700741B2FF582E43402F583E4F012D54F22F7
:10B12D000A4845494748540A43414C494252415403
:10B13D00494F4E000A414E474C450A43414C494246
:10B14D00524154494F4E000A5349440A43414C4918
:10B15D0042524154494F4E000A4445544543544FC1
:10B16D005220524F540A43414C4942524154494F87
:10B17D004E0025732573000A0A352D454E54455250
:10B18D000A342D4C4556454C2055500A362D4C450C
:10B19D0056454C20444F574E0A312B322B332051FC
:10B1AD0055495400502531642E2531642573000A0C
:10B1BD000A505245535320312B3320544F20414CCC
:10B1CD004C4F57204D4F56454D454E540A0A342D80
:10B1DD005355424C4556454C2055500A362D535526
:10B1ED00424C4556454C20444F574E0A0A352D5179
:10B1FD005549540000010158210101C80201015AAD
:10B20D00210101C80401015C210101C8FF000000FA
:10B21D00010000000601015E0101018608010160C7
:10B22D00010101860A010162010101860C0101641F
:10B23D0001010186FF000000010000000E01016602
:10B24D002101013F100101682101013FFF000000B4
:10B25D00010000001201016A210101231401016C9A
:10B26D00210101231601016E21010123FF000000C0
:10B27D0001000000FFB201FFB221FFB249FFB26130
:0CB28D00FFB12DFFB141FFB154FFB165CE
:0EDF7500E4900288F0900287F0900286F0227D
:10D93B00900288E075F003A42481F582E434B2F5FB
:10D94B0083E493FB740193FA740293F9900287E0DA
:10D95B0075F008A4FFE92FF9EA35F0FAE92408F984
:0CD96B00E43AFA122CC7F46002D322C385
:01D97700228D
:10DC3000900286E0700DA3F0A3E0C39403500FE0C0
:0FDC400004F02212D93B5006900287E004F02234
:10DD6800900286E07009A3F0A3E0600B14F0229003
:08DD78000287E0600214F022B2
:10DF3700900286E06003E4F02290028674FFF022EC
:07E03000900286E024FF22AC
:10C76C00900288E075F003A42481F582E434B2F5DC
:10C77C0083E493FB740193FA740293F9900287E0BB
:10C78C0075F008A4FFE92FF9EA35F0FA9000D0EB28
:10C79C00F0A3EAF0A3E9F0122CC7FFC3139000D367
:10C7AC00F0A37401F0A37401F0A3749CF09000D377
:10C7BC00E075F002A4FF9000D5E5F08FF0122DBCCF
:10C7CC009000D0E0FBA3E0FAA3E0F9900005123052
:10C7DC005F122DD2FF9000D4E0FBA3E0FAA3E0F9A6
:10C7EC00E5F08FF0122E359000D3E0FFA3E0FBA311
:08C7FC00E0FAA3E0F912D5EF09
:01C804002211
:10D68E00900288E075F003A42481F582E434B2F5AB
:10D69E0083E493FB740193FA740293F9900287E08A
:10D6AE0075F008A4FFE92FF9EA35F0FA122CC7FF3E
:10D6BE00C313FF7B017A01799C75F002A429F9E569
:09D6CE00F03AFA122DD2FFAEF081
:01D6D7002230
:10C06600900288E0122D40900287E0FF9000D3E016
:10C07600FBA3E0FAA3E0F9EF122D40900286E0FF61
:10C086009000D6E0FBA3E0FAA3E0F9EF122D409072
:10C096000286E0704F9000EB74FFF0A374B1F0A33A
:10C0A600747FF0900288E075F003A4248DF582E495
:10C0B60034B2F583E493F9740193FA740293900011
:10C0C600EEC9F0A3EAF0A3E9F0A374FFF0A374B1FC
:10C0D600F0A37484F09000D9E0FBA3E0FAA3E0F9A2
:10C0E600126C13229000EB74FFF0A374B1F0A374EA
:10C0F600B1F0900288E02401FEE4339000EEF0A354
:10C10600CEF0900287E02401FEE4339000F0F0A325
:10C11600CEF0A374FFF0A374B1F0A374BCF090004A
:0DC12600D9E0FBA3E0FAA3E0F9126C1322AC
:0BCC8400900008EBF0A3EAF0A3E9F039
:10CC8F00900288E075F003A42481F582E434B2F5B4
:10CC9F0083E493FB740193FA740293F9900287E093
:10CCAF0075F008A4FFE92FF9EA35F0FA90000EEBC2
:10CCBF00F0A3EAF0A3E9F090000112305F122DD239
:10CCCF00FF900008E0FBA3E0FAA3E0F9E5F08FF096
:10CCDF00122E3590000EE0FBA3E0FAA3E0F99000CE
:10CCEF0004122CE0FF90000BE0FBA3E0FAA3E0F9A5
:04CCFF00EF122D40C3
:01CD0300220D
:1074A7000020434D00494E43004D535700504F5461
:1074B70000302D434D0A312D494E43484553000AAC
:1074C700524F4F4D204D4158204845494748540099
:1074D7000A54484F52415820484549474854005597
:1074E7004E4445525441424C45204845494748542B
:1074F700000A5441424C4520484549474854000A30
:107507004445544543544F52204845494748540041
:107517004445544543544F522057494454482D4CF1
:10752700454654004445544543544F522057494417
:1075370054482D524947485400544849524420530F
:10754700494420504F534954494F4E0053454355E2
:10755700524954592044495354414E4345005448D5
:107567004F52415820534944000A4D494E2048453F
:1075770049474854000A4D4158204845494748540F
:10758700000A48414C462057415920484549474839
:1075970054000A4D494E20414E474C45000A564576
:1075A70052544943414C20414E474C4500484F52A5
:1075B700495A4F4E54414C20414E474C45000A4DC5
:1075C700415820414E474C45000A4D494E205349EA
:1075D70044000A4D415820534944000A4D494E2062
:1075E7004445544543544F5220524F54000A444592
:1075F70054454E54204445544543544F52000A4D78
:107607004158204445544543544F5220524F54004B
:107617000A47454E4552414C0A53455454494E4733
:1076270053000A47454E4552414C0A534554544965
:107637004E47532032000A4845494748540A5345A4
:107647005454494E4753000A414E474C450A534547
:107657005454494E4753000A5349440A5345545416
:10766700494E4753000A4445544543544F5220520C
:107677004F540A53455454494E47530025732573B5
:10768700000A0A352D454E5445520A342D4C4556AD
:10769700454C2055500A362D4C4556454C20444FF5
:1076A700574E0A312B322B332051554954000A0AC1
:1076B700312D56414C55452055500A332D56414CD6
:1076C700554520444F574E0A322D534156452056B3
:1076D700414C55450A342D5355424C4556454C208F
:1076E70055500A362D5355424C4556454C20444F6C
:1076F700574E0A352D5155495400FF74A7FF74A8FA
:10770700FF74ACFF74B0FF74B4000000000101FF08
:1077170074B8000200F0015E21FF74C6000400285F
:1077270000F021FF74D70006000F009621FF74E6D2
:107737000008002800F021FF74F8000A000A003C46
:1077470021FF7506000C001E009621FF7517000E1D
:10775700000A009621FF752B0010000000FA21FF98
:10776700754000FF0000000001FF770100120005CF
:10777700001E21FF75530014000000FA21FF7565F4
:1077870000FF0000000001FF77010016002800F04D
:1077970021FF75700018002800F021FF757C001A82
:1077A700002800F021FF758800FF0000000001FF9E
:1077B7007701001CFFA600B401FF7599001EFFA604
:1077C70000B401FF75A40020FFA600B401FF75B443
:1077D7000022FFA600B401FF75C500FF00000000EE
:1077E70001FF77010024000000FA21FF75D0002671
:1077F700000000FA21FF75D900FF0000000001FF1B
:1078070077010028FFA6005A01FF75E2002AFFA6AC
:10781700005A01FF75F4002CFFA6005A01FF7605F8
:1078270000FF0000000001FF770100FF7710FF77DE
:1078370074FF7792FF77BAFF77ECFF780AFF761726
:0F784700FF7629FF763DFF764EFF765EFF766C6B
:10D4FE00900285E075F003A42432F582E43478F5C9
:10D50E0083E493FB740193FA740293F9900282E020
:10D51E0075F00AA4FFE92FF9EA35F0FA122CC7FFCD
:10D52E00C313FF7B017A01794275F002A429F9E554
:10D53E00F03AFA122DD2FF900283E5F0F0A3EFF04D
:01D54E0022BA
:10DEF400E4900285F0900282F0900281F012D4FE48
:01DF040022FA
:10D76A00900285E075F003A42432F582E43478F55A
:10D77A0083E493FB740193FA740293F9900282E0B2
:10D78A0075F00AA4FFE92FF9EA35F0FAE9240AF953
:10D79A00E43AFA122CC7F4600D900009122CE060EA
:07D7AA0003300E02D322C37D
:01D7B1002255
:10DB6300900281E07010A3F0900285E0C394055009
:10DB730010E004F0800B12D76A5006900282E00492
:05DB8300F012D4FE22A7
:10DCAC00900281E0700CA3F0900285E0600C14F0FF
:0EDCBC008008900282E0600214F012D4FE2272
:10DE5C00900281E06004E4F0800690028174FFF08F
:04DE6C0012D4FE22AC
:06E04500900281E0FF22C1
:10D40300900285E075F003A42432F582E43478F5C4
:10D4130083E493FB740193FA740293F9900282E01C
:10D4230075F00AA4FFE92FF9EA35F0FA9000031228
:10D433002DFDFFC3900284E09FE5F06480F8900225
:10D4430083E0648098500CA3E004F070069002839C
:03D45300E004F002
:01D4560022B3
:10D45700900285E075F003A42432F582E43478F570
:10D4670083E493FB740193FA740293F9900282E0C8
:10D4770075F00AA4FFE92FF9EA35F0FA90000112D6
:10D487002DFDFFD3900284E09FE5F06480F89002C1
:10D4970083E0648098400CA3E024FFF0900283E0CF
:03D4A70034FFF05F
:01D4AA00225F
:10D29D00900285E075F003A42432F582E43478F52C
:10D2AD0083E493FB740193FA740293F9900282E084
:10D2BD0075F00AA4FFE92FF9EA35F0FA122CC7FF31
:10D2CD00C313900005F07B017A017942E075F002FD
:10D2DD00A429F9E5F03AFA900283E0FFA3E0CF8F9D
:0CD2ED00F0122E35900005E0FF12D59FD6
:01D2F9002212
:0BA992009000D3EBF0A3EAF0A3E9F083
:10A99D00900281E0601A900283E0F9A3E0FF90003D
:10A9AD00DCE0FBA3E0FAA3E0C98FF0122E35801195
:10A9BD009000DCE0FBA3E0FAA3E0F9E4F5F0122E41
:10A9CD0035900285E075F003A42432F582E43478E5
:10A9DD00F583E493FB740193FA740293F990028268
:10A9ED00E075F00AA4FFE92FF9EA35F0FA9000E5D9
:10A9FD00EBF0A3EAF0A3E9F0900285E0FF9000D31D
:10AA0D00E0FBA3E0FAA3E0F9EF122D40900282E003
:10AA1D00FF9000D6E0FBA3E0FAA3E0F9EF122D4082
:10AA2D00900281E0FF9000D9E0FBA3E0FAA3E0F9EA
:10AA3D00EF122D409000E5E0FBA3E0FAA3E0F990C2
:10AA4D000005122CE0FF9000DFE0FBA3E0FAA3E08D
:10AA5D00F9EF122D40900281E0704F9000EB74FFE2
:10AA6D00F0A37476F0A37483F0900285E075F00383
:10AA7D00A42444F582E43478F583E493F9740193C6
:10AA8D00FA7402939000EEC9F0A3EAF0A3E9F0A3E3
:10AA9D0074FFF0A37476F0A37488F09000E2E0FBED
:10AAAD00A3E0FAA3E0F9126C13229000E5E0FBA3FA
:10AABD00E0FAA3E0F990000612305F74FF90770181
:10AACD006B7008E965827003EA658360449000EB62
:10AADD0074FFF0A37476F0A37483F09000E5E0FBAF
:10AAED00A3E0FAA3E0F990000612305F9000EEEBC0
:10AAFD00F0A3EAF0A3E9F0A374FFF0A37476F0A33A
:10AB0D0074B5F09000E2E0FBA3E0FAA3E0F9126C5B
:01AB1D001324
:01AB1E002214
:0CDFEB006000010750000107400000002A
:10D97800C2AFEF25E025E024EBF582E434DFF58340
:10D98800E493FE7401937810A60608F6D297ED4446
:10D9980038FF18E6FC08E6FDF5828C83EFF0C297A5
:0CD9A8009000F4E04B8D828C83F0D2AF35
:01D9B4002250
:0AD9EF0090000CEFF0A3EBF0A90587
:10D9F900AA0190000DE0FFE92FFFE433FEEAC39F7F
:10DA0900EE6480F8748098501590000CE0FFAD0228
:0EDA19009000F47480F0E4FB12D9780A80D4F7
:01DA270022DC
:10D63F009000EAEFF0A3EDF0A3EBF0A3EAF0A3E97B
:01D64F00F0EA
:10D65000E49000F0F09000EFE0FFA3E0FEC39F50E5
:10D660002C9000EAE0FFA3E02EFDA3E0FBA3E0FA8C
:10D67000A3E0F98E82758300122CE0FB9000F47415
:0DD6800080F012D9789000F0E004F080C82E
:01D68D00227A
:10CD8000E4900008F0900008E0FFC394035068EFBF
:10CD900025E025E024EEF582E434DFF583E493908A
:10CDA0000009F0900008E0FF25E025E024EDF58281
:10CDB000E434DFF583E493FDEF25E025E024EEF590
:10CDC00082E434DFF583E4932DFFE433FE90000921
:10CDD000E0FDC39FEE6480F87480985012900008C4
:10CDE000E0FFE4FB12D87F900009E004F080B490EB
:07CDF0000008E004F0808E52
:01CDF7002219
:10D87F00EB30E705547FFB8004EB4480FBC2AFEF36
:10D88F0025E025E024EBF582E434DFF583E493FE15
:10D89F007401937810A60608F6D297ED4438FF1856
:10D8AF00E6FC08E6F5828C83EFF0C297EBF0D2AF7F
:01D8BF002246
:0300030002C57FB4
:10C57F00C0E0C0F0C083C082C0D075D000C000C082
:10C58F0001C002C003C004C005C006C00720B26EC0
:10C59F00C2A8C2AA9001C6E05408FF90018FE054D0
:10C5AF00204FFF90013CE054044F900183F0C39063
:10C5BF000184E0648094805012900183E0FF900129
:10C5CF0020E05410FEEF4E900183F0C2057F3F1222
:10C5DF00DBD0C2057F0312DC10900120E4F0900144
:10C5EF008FF09001C7F090019BF09001C6F0900181
:10C5FF003CF090017574FFF09001887408F0D0073B
:10C60F00D006D005D004D003D002D001D000D0D0B6
:09C61F00D082D083D0F0D0E032CB
:0300130002C4D054
:10C4D000C0E0C0F0C083C082C0D075D000C000C032
:10C4E00001C002C003C004C005C006C00720B37469
:10C4F000C2AAC2A89001C6E05408FF90018FE05480
:10C50000204FFF90013CE054044F900183F0C39012
:10C510000185E09432900184E06480948050129010
:10C520000183E0FF900120E05410FEEF4E90018364
:10C53000F0C2057F3F12DBD0C2057F0312DC1090F2
:10C540000120E4F090018FF09001C7F090019BF082
:10C550009001C6F090013CF090017674FFF09001DC
:10C56000887408F0D007D006D005D004D003D002DC
:0FC57000D001D000D0D0D082D083D0F0D0E03234
:10BB6500E4900137F012DDC6E4900138F012DDDC17
:10BB7500E4900139F012DDF2C204C205C206C20723
:10BB8500C208E4900008F0C209D20A12CC01C2042E
:10BB950012C6CA7F5B12DFF7C204D205D206C207FE
:10BBA500C208E4900008F0C209D20A12CC01C2040E
:10BBB50012C6CAC2047F0112DCCAC20412C6CA1266
:10BBC500000EE4FF12DFF7C20412D6D8AC06AD07AB
:10BBD5007F0112D23EC204E4FF12DCCAC20412C6BF
:10BBE500CA12000EE4FF12DFF7C20412D6D8AC0663
:10BBF500AD07E4FF12D23EC2047F0212DCCAC204C2
:10BC050012C6CA12000EE4FF12DFF7C20412D6D81C
:10BC1500AC06AD077F0212D23EC2047F0312DCCA16
:10BC2500C20412C6CA12000EE4FF12DFF7C20412E4
:0CBC3500D6D8AC06AD077F0312D23E2229
:10DE0800C2AF7580FF7835E6FE08E6F5828E83E0BE
:04DE1800F4FFD2AF92
:01DE1C0022E3
:10DE1D00C2AF7580FF782FE6FE08E6F5828E83E0AF
:04DE2D00F4FFD2AF7D
:01DE310022CE
:10DE3200C2AF7580FF7831E6FE08E6F5828E83E098
:04DE4200F4FFD2AF68
:01DE460022B9
:10DBD000AD07C2AF300508900137E04FF0800B90E1
:10DBE0000137E0FFEDF4FEEF5EF012DDC6D2AF22AA
:10DBF000AD07C2AF300408900138E04FF0800B90C1
:10DC00000138E0FFEDF4FEEF5EF012DDDCD2AF2272
:10DC1000AD07C2AF300508900139E04FF0800B909E
:10DC20000139E0FFEDF4FEEF5EF012DDF2D2AF223B
:10DDC600C2AF900137E0FF7825E6FC08E6F5828CC5
:06DDD60083EFF0D2AF2242
:10DDDC00C2AF900138E0FF7829E6FC08E6F5828CAA
:06DDEC0083EFF0D2AF222C
:10DDF200C2AF900139E0FF782BE6FC08E6F5828C91
:06DE020083EFF0D2AF2215
:10A2C600E4900007F09001A4E0FEA3E0FFC3900134
:10A2D600A3E09FEE6480F89001A2E0648098503578
:10A2E600900007E0FF25E024A2F582E43401F5831F
:10A2F600E0FCA3E0FDD3900187E09DEC6480F8903C
:10A306000186E06480984043EF9404503E90000735
:10A31600E004F080CB900007E0FF25E024A2F58260
:10A32600E43401F583E0FCA3E0FDC3900187E09DE2
:10A33600EC6480F8900186E0648098500EEFC39438
:10A34600045008900007E004F080CA900007E0FF80
:10A356007005E004F0800AEFB40406900007E014EC
:10A36600F0900007E025E024A0F582E43401F583AF
:10A37600E0FCA3E0FDEC122918900008122FE290F1
:10A386000007E025E0245CF582E43401F583E0FC77
:10A39600A3E0FDEC122918900010122FE29000079E
:10A3A600E025E024A2F582E43401F583E0FCA3E095
:10A3B600FDEC12291890000C122FE2900007E02500
:10A3C600E0245EF582E43401F583E0FCA3E0FDECD5
:10A3D600122918900014122FE2900186E0FCA3E0E7
:10A3E600FDEC122918900008E0F8A3E0F9A3E0FAC2
:10A3F600A3E0FB122678C004C005C006C007900083
:10A4060010E0F8A3E0F9A3E0FAA3E0FBA3E0FCA3C5
:10A41600E0FDA3E0FEA3E0FF122678D003D002D031
:10A4260001D00012276DC004C005C006C007900009
:10A4360008E0F8A3E0F9A3E0FAA3E0FBA3E0FCA39D
:10A44600E0FDA3E0FEA3E0FF122678A804A905AA72
:10A4560006AB07D007D006D005D0041228769000A8
:10A4660010E0F8A3E0F9A3E0FAA3E0FB12267C12C1
:0AA476002951900184EEF0A3EFF0ED
:01A4800022B9
:10A48100E4900007F09001B0E0FEA3E0FFC390016B
:10A49100AFE09FEE6480F89001AEE06480985035A3
:10A4A100900007E0FF25E024AEF582E43401F58356
:10A4B100E0FCA3E0FDD3900124E09DEC6480F890E2
:10A4C1000123E06480984043EF9403503E900007DD
:10A4D100E004F080CB900007E0FF25E024AEF58298
:10A4E100E43401F583E0FCA3E0FDC3900124E09D89
:10A4F100EC6480F8900123E0648098500EEFC394DF
:10A50100035008900007E004F080CA900007E0FFC4
:10A511007005E004F0800AEFB40306900007E01430
:10A52100F0900007E025E024ACF582E43401F583E6
:10A53100E0FCA3E0FDEC122918900008122FE29034
:10A541000007E025E02468F582E43401F583E0FCAE
:10A55100A3E0FDEC122918900010122FE2900007E1
:10A56100E025E024AEF582E43401F583E0FCA3E0CC
:10A57100FDEC12291890000C122FE2900007E02543
:10A58100E0246AF582E43401F583E0FCA3E0FDEC0C
:10A59100122918900014122FE2900123E0FCA3E08D
:10A5A100FDEC122918900008E0F8A3E0F9A3E0FA05
:10A5B100A3E0FB122678C004C005C006C0079000C6
:10A5C10010E0F8A3E0F9A3E0FAA3E0FBA3E0FCA309
:10A5D100E0FDA3E0FEA3E0FF122678D003D002D075
:10A5E10001D00012276DC004C005C006C00790004D
:10A5F10008E0F8A3E0F9A3E0FAA3E0FBA3E0FCA3E1
:10A60100E0FDA3E0FEA3E0FF122678A804A905AAB5
:10A6110006AB07D007D006D005D0041228769000EB
:10A6210010E0F8A3E0F9A3E0FAA3E0FB12267C1204
:0AA631002951900121EEF0A3EFF093
:01A63B0022FC
:10A63C00E4900007F09001ACE0FEA3E0FFC39001B2
:10A64C00ABE09FEE6480F89001AAE06480985035EE
:10A65C00900007E0FF25E024AAF582E43401F5839D
:10A66C00E0FCA3E0FDD3900140E09DEC6480F89009
:10A67C00013FE06480984043EF9402503E90000705
:10A68C00E004F080CB900007E0FF25E024AAF582DF
:10A69C00E43401F583E0FCA3E0FDC3900140E09DB0
:10A6AC00EC6480F890013FE0648098500EEFC39406
:10A6BC00025008900007E004F080CA900007E0FF09
:10A6CC007005E004F0800AEFB40206900007E01475
:10A6DC00F0900007E025E024A8F582E43401F5832E
:10A6EC00E0FCA3E0FDEC122918900008122FE29078
:10A6FC000007E025E02464F582E43401F583E0FCF6
:10A70C00A3E0FDEC122918900010122FE290000724
:10A71C00E025E024AAF582E43401F583E0FCA3E013
:10A72C00FDEC12291890000C122FE2900007E02586
:10A73C00E02466F582E43401F583E0FCA3E0FDEC53
:10A74C00122918900014122FE290013FE0FCA3E0B4
:10A75C00FDEC122918900008E0F8A3E0F9A3E0FA48
:10A76C00A3E0FB122678C004C005C006C007900009
:10A77C0010E0F8A3E0F9A3E0FAA3E0FBA3E0FCA34C
:10A78C00E0FDA3E0FEA3E0FF122678D003D002D0B8
:10A79C0001D00012276DC004C005C006C007900090
:10A7AC0008E0F8A3E0F9A3E0FAA3E0FBA3E0FCA324
:10A7BC00E0FDA3E0FEA3E0FF122678A804A905AAF9
:10A7CC0006AB07D007D006D005D00412287690002F
:10A7DC0010E0F8A3E0F9A3E0FAA3E0FB12267C1248
:0AA7EC002951900173EEF0A3EFF085
:01A7F6002240
:10909D00E4900007F090019EE0FEA3E0FFC3900175
:1090AD009DE09FEE6480F890019CE06480985035BF
:1090BD00900007E0FF25E0249CF582E43401F58360
:1090CD00E0FCA3E0FDD39001C9E09DEC6480F89035
:1090DD0001C8E06480984043EF9403503E90000730
:1090ED00E004F080CB900007E0FF25E0249CF582A2
:1090FD00E43401F583E0FCA3E0FDC39001C9E09DDC
:10910D00EC6480F89001C8E0648098500EEFC39431
:10911D00035008900007E004F080CA900007E0FFBC
:10912D007005E004F0800AEFB40306900007E01428
:10913D00F0900007E025E0249AF582E43401F583F0
:10914D00E0FCA3E0FDEC122918900008122FE2902C
:10915D000007E025E02456F582E43401F583E0FCB8
:10916D00A3E0FDEC122918900010122FE2900007D9
:10917D00E025E0249CF582E43401F583E0FCA3E0D6
:10918D00FDEC12291890000C122FE2900007E0253B
:10919D00E02458F582E43401F583E0FCA3E0FDEC16
:1091AD00122918900014122FE29001C8E0FCA3E0E0
:1091BD00FDEC122918900008E0F8A3E0F9A3E0FAFD
:1091CD00A3E0FB122678C004C005C006C0079000BE
:1091DD0010E0F8A3E0F9A3E0FAA3E0FBA3E0FCA301
:1091ED00E0FDA3E0FEA3E0FF122678D003D002D06D
:1091FD0001D00012276DC004C005C006C007900045
:10920D0008E0F8A3E0F9A3E0FAA3E0FBA3E0FCA3D8
:10921D00E0FDA3E0FEA3E0FF122678A804A905AAAD
:10922D0006AB07D007D006D005D0041228769000E3
:10923D0010E0F8A3E0F9A3E0FAA3E0FB12267C12FC
:10924D002951900170EEF0A3EFF0900184E0FEA3A0
:10925D00E0FF900121E0FCA3E0FD1261FE900018FB
:10926D00EEF0A3EFF0900184E0FEA3E0FF9001216A
:10927D00E0FCA3E0FD1266F6900170E0FCA3E0FDBA
:10928D00D39FEE6480F8EC648098401DED24FEFDC4
:10929D00EC34FFFCD3ED9FEE6480F8EC64809850C5
:1092AD0008900170EEF0A3EFF0900018E0FEA3E03F
:1092BD00FF900170E0FCA3E0FDC39FEE6480F8EC2D
:1092CD006480985022ED2402FDE43CFCD3EF9DEC2C
:1092DD006480F8EE648098500E900018E0A3E09042
:0792ED000170EEF0A3EFF0A9
:0192F4002257
:0E61FE00900030EEF0A3EFF0A3ECF0A3EDF074
:10620C00E4A3F0A3F0A3F0A3F0A3F0A3F0A3F0A3F6
:10621C00F0A3F0900047F0A3F0FBFAED2FFFEC3E5B
:10622C00900041F0A3EFF0900030E0FEA3E0FFD32C
:10623C00945AEE64809480400974B49FFBE49EFAF7
:10624C008008900030E0FAA3E0FBAE02AF03AD078C
:10625C00AC06EC1229187BC37AF5794878401227E2
:10626C006DE4FBFA7934784312287690003D122FB6
:10627C00E2900041E0FCA3E0FDEC1229187BC37A0C
:10628C00F57948784012276DE4FBFA79347843129B
:10629C002876900043122FE290003DE0FCA3E0FD35
:1062AC00A3E0FEA3E0FF12ACF0E4FBFA79DC784249
:1062BC0012276D122951900035EEF0A3EFF0FDACD2
:1062CC0006EC12291812DFDE122951900035EEF07F
:1062DC00A3EFF090003DE0FCA3E0FDA3E0FEA3E003
:1062EC00FF12ACF0E4FBFA79B4784212276D122954
:1062FC0051900037EEF0A3EFF0FDAC06EC1229182C
:10630C0012DFDE122951900037EEF0A3EFF090006F
:10631C0030E0FEA3E0FFD3945AEE64809480500BDF
:10632C00C3900041E064809480401FD3EF945AEEF8
:10633C0064809480405C900041E0FEA3E0FF74B464
:10634C009FE49EC3648094805048900043E0FCA37B
:10635C00E0FDA3E0FEA3E0FF12AD06C004C005C043
:10636C0006C00790014EE0FCA3E0FDEC12291812C8
:10637C002951AD07AC06EC122918D003D002D0017C
:10638C00D00012276D122951900039EEF0A3EFF0D6
:10639C008046900043E0FCA3E0FDA3E0FEA3E0FFF9
:1063AC0012AD06C004C005C006C007900150E0FC49
:1063BC00A3E0FDEC122918122951AD07AC06EC1222
:1063CC002918D003D002D001D00012276D12295108
:1063DC00900039EEF0A3EFF0900039E0FCA3E0FD63
:1063EC00EC12291812DFDE122951900039EEF0A3BD
:1063FC00EFF0900030E0FEA3E0FFC3945AEE64800F
:10640C0094805011C3900042E0945A900041E06493
:10641C008094804028C3EF945AEE6480948050039B
:10642C000264B1900041E0FEA3E0FF74B49FFFE46E
:10643C009EFEC3EF945AEE648094804068900043B3
:10644C00E0FCA3E0FDA3E0FEA3E0FF12ACF0C0046F
:10645C00C005C006C00790014CE0FCA3E0FDEC12A7
:10646C002918122951AD07AC06EC122918D003D00B
:10647C0002D001D00012276D12DFDEC004C005C0AF
:10648C0006C007900039E0FCA3E0FDEC122918D0FF
:10649C0003D002D001D00012267C12295190003971
:1064AC00EEF0A3EFF0D3900174E09496900173E0BA
:1064BC00648094804045900188E06406603D9000C3
:1064CC003DE0FCA3E0FDA3E0FEA3E0FF12AD06E47B
:1064DC00FBFA79F0784112276D12295190003BEEAE
:1064EC00F0A3EFF0FDAC06EC12291812DFDE122936
:1064FC005190003BEEF0A3EFF0803B90003DE0FCB0
:10650C00A3E0FDA3E0FEA3E0FF12AD06E4FBFA79E5
:10651C0070784112276D12295190003BEEF0A3EFD9
:10652C00F0FDAC06EC12291812DFDE122951900096
:10653C003BEEF0A3EFF0C3900031E0945A900030A2
:10654C00E064809480505C900037E0FEA3E0FF9004
:10655C00003AE02FFF900039E03EFE900035E0FC61
:10656C00A3E0FDC390003CE09DFD90003BE09CFC53
:10657C00D3ED9FEE6480F8EC648098400A9000475D
:10658C00ECF0A3EDF08077900037E0FEA3E0FF90F5
:10659C00003AE02FFF900039E03E900047F0A3EF67
:1065AC00F0805B900037E0FEA3E0FFC390003AE080
:1065BC009FFF900039E09EFE900035E0FCA3E0FDCB
:1065CC0090003CE02DFD90003BE03CFCD3ED9FEEB9
:1065DC006480F8EC648098400A900047ECF0A3EDDE
:1065EC00F0801B900037E0FEA3E0FFC390003AE080
:1065FC009FFF900039E09E900047F0A3EFF09001D0
:10660C0054E0FEA3E0FF900048E02FF0900047E03C
:10661C003EF0900158E0FEA3E0FFC3900048E09FDD
:10662C00EE6480F8900047E064809840629001210D
:10663C00E0FEA3E0FF900032E06E7003A3E06F7009
:10664C005D900184E0FCA3E0FD900030E06C7003F1
:10665C00A3E06D7049D3ED945BEC64809480503E64
:10666C00C3ED9459EC648094804033D3EF9401EEE5
:10667C00648094805028C3900122E094FF90012103
:10668C00E06480947F4017900188E06406600F906E
:10669C000158E0FFA3E0900047CFF0A3EFF0D390B8
:1066AC000185E09400900184E06480948040327F06
:1066BC000B12C92FEF640160087F0B12C92FBF02A8
:1066CC002090014AE0FEA3E0FFC3900048E09FEE5B
:1066DC006480F8900047E06480985005EEF0A3EFDA
:0966EC00F0900047E0FEA3E0FF7E
:0166F5002282
:1066F600900032ECF0A3EDF0900030EEF0A3EFF056
:10670600E4900034F0FDFCA3F0A3F0A3F0A3F0A303
:10671600F0A3F0A3F0A3F0900047F0A3F0FBFAD3A8
:10672600EF945AEE648094804011900030E0FEA30E
:10673600E0FF74B49FFBE49EFA8008900030E0FA14
:10674600A3E0FBAE02AF03AD07AC06EC1229187B43
:10675600C37AF57948784012276DE4FBFA793478E4
:106766004312287690003D122FE2900030E0FEA3FF
:10677600E0FF900033E02FFF900032E03EFE9000F5
:1067860041F0A3EFF0FDAC06EC1229187BC37AF5B5
:106796007948784012276DE4FBFA79347843122859
:1067A60076900043122FE290003DE0FCA3E0FDA3AB
:1067B600E0FEA3E0FF12ACF0E4FBFA79DC784212CB
:1067C600276D122951900035EEF0A3EFF0FDAC06CF
:1067D600EC12291812DFDE122951900035EEF0A3D3
:1067E600EFF090003DE0FCA3E0FDA3E0FEA3E0FF98
:1067F60012ACF0E4FBFA79B4784212276D122951F3
:10680600900037EEF0A3EFF0FDAC06EC122918125B
:10681600DFDE122951900037EEF0A3EFF090003042
:10682600E0FEA3E0FFD39400EE6480948050030260
:106836006907900041E0FCA3E0FDD39400EC64807E
:106846009480400BD3EF945AEE648094804024C326
:1068560074B49DFFE49CFED3EF9400EE64809480B4
:106866004059D3900031E0945A900030E06480940F
:10687600804048900043E0FCA3E0FDA3E0FEA3E0D7
:10688600FF12AD06C004C005C006C00790014EE069
:10689600FCA3E0FDEC122918122951AD07AC06EC59
:1068A600122918D003D002D001D00012276D122968
:1068B60051900039EEF0A3EFF08046900043E0FCE3
:1068C600A3E0FDA3E0FEA3E0FF12AD06C004C005F1
:1068D600C006C007900150E0FCA3E0FDEC122918A9
:1068E600122951AD07AC06EC122918D003D002D0FC
:1068F60001D00012276D122951900039EEF0A3EF56
:10690600F0900039E0FCA3E0FDEC12291812DFDE5E
:10691600122951900039EEF0A3EFF0900030E0FE1E
:10692600A3E0FFD3945AEE648094805011C3900084
:1069360042E0945A900041E0648094805028D3EF5E
:10694600945AEE6480948050030269D4900041E02A
:10695600FEA3E0FF74B49FFFE49EFEC3EF945AEEDD
:10696600648094805068900043E0FCA3E0FDA3E0BF
:10697600FEA3E0FF12ACF0C004C005C006C007903D
:10698600014CE0FCA3E0FDEC122918122951AD07D9
:10699600AC06EC122918D003D002D001D000122781
:1069A6006D12DFDEC004C005C006C007900039E0E6
:1069B600FCA3E0FDEC122918D003D002D001D000D0
:1069C60012267C122951900039EEF0A3EFF0D390F5
:1069D6000174E09496900173E06480948040459041
:1069E6000188E06406603D90003DE0FCA3E0FDA365
:1069F600E0FEA3E0FF12AD06E4FBFA79F07841125F
:106A0600276D12295190003BEEF0A3EFF0FDAC0686
:106A1600EC12291812DFDE12295190003BEEF0A38A
:106A2600EFF0803B90003DE0FCA3E0FDA3E0FEA379
:106A3600E0FF12AD06E4FBFA7970784112276D1279
:106A4600295190003BEEF0A3EFF0FDAC06EC1229C5
:106A56001812DFDE12295190003BEEF0A3EFF0C3CF
:106A6600900031E0945A900030E064809480507534
:106A7600900037E0FEA3E0FFC390003AE09FFF904E
:106A86000039E09EFE900035E0FCA3E0FD90003C5E
:106A9600E02DFD90003BE03CFCD3ED9FEE6480F8DA
:106AA600EC6480984015900145E09DFE900144E01D
:106AB6009C900047F0A3CEF0026B5C900037E0FE9E
:106AC600A3E0FFC390003AE09FFF900039E09EFEEE
:106AD600C3900145E09FFF900144E09E900047F07F
:106AE600A3EFF08071900037E0FEA3E0FF90003A3C
:106AF600E02FFF900039E03EFE900035E0FCA3E079
:106B0600FDC390003CE09DFD90003BE09CFCD3ED76
:106B16009FEE6480F8EC6480984014900145E09DF7
:106B2600FE900144E09C900047F0A3CEF0802790B1
:106B36000037E0FEA3E0FF90003AE02FFF90003917
:106B4600E03EFEC3900145E09FFF900144E09E9029
:106B56000047F0A3EFF0900048E024FBF0900047D8
:106B6600E034FFF0900184E0FEA3E0FF900030E007
:106B76006E7003A3E06F6007900188E0B406209072
:106B8600015AE0FEA3E0FFD3900048E09FEE648048
:106B9600F8900047E06480984005EEF0A3EFF0908F
:076BA6000047E0FEA3E0FF41
:016BAD0022C5
:10CDF800E4900030F0A3F0FDFCD3EF945AEE648089
:10CE08009480400974B49FFDE49EFC8004AC06AD98
:10CE180007AE04AF05EC1229187BC37AF579487878
:10CE28004012276DE4FBFA7934784312287612AC65
:10CE3800F0E4FBFA79B4784212276D122951900078
:10CE480030EEF0A3EFF0FDAC06EC12291812DFDE8D
:10CE5800122951900030EEF0A3EFF0900149E02F35
:07CE6800FF900148E03EFECF
:01CE6F0022A0
:109F3C00C2047F0112DCCAC20412C6CA12000EE4AB
:109F4C00FF12DFF7C20412D6D8AC06AD077F0112A0
:109F5C00B75C900005EEF0A3EFF09001C8E0FCA315
:109F6C00E0FD2403FBE43CFAD3EB9FEE6480F8EABB
:109F7C00648098401BED24FDFFEC34FFFED3900071
:109F8C0006E09FEE6480F8900005E0648098500F26
:109F9C00900005E0FFA3E09001C8CFF0A3EFF0C262
:109FAC0004E4FF12DCCAC20412C6CA12000EE4FF9B
:109FBC0012DFF7C20412D6D8AC06AD07E4FF12B715
:109FCC005C900005EEF0A3EFF0900186E0FCA3E0BE
:109FDC00FD2403FBE43CFAD3EB9FEE6480F8EA64C7
:109FEC008098401BED24FDFFEC34FFFED39000065F
:109FFC00E09FEE6480F8900005E0648098500F902C
:10A00C000005E0FFA3E0900186CFF0A3EFF0C204BF
:10A01C007F0212DCCAC20412C6CA12000EE4FF127E
:10A02C00DFF7C20412D6D8AC06AD077F0212B75CBC
:10A03C00900005EEF0A3EFF090013FE0FCA3E0FDF3
:10A04C002403FBE43CFAD3EB9FEE6480F8EA6480D3
:10A05C0098401BED24FDFFEC34FFFED3900006E08E
:10A06C009FEE6480F8900005E0648098500F90009B
:10A07C0005E0FFA3E090013FCFF0A3EFF0C2047F17
:10A08C000312DCCAC20412C6CA12000EE4FF12DFAD
:10A09C00F7C20412D6D8AC06AD077F0312B75C909A
:10A0AC000005EEF0A3EFF0900123E0FCA3E0FD240B
:10A0BC0003FBE43CFAD3EB9FEE6480F8EA648098EF
:10A0CC00401BED24FDFFEC34FFFED3900006E09F17
:10A0DC00EE6480F8900005E0648098500F900005C5
:10A0EC00E0FFA3E0900123CFF0A3EFF012A2C61281
:08A0FC00A63C12909D12A48104
:01A104002238
:10AB1F00202020004B4559424F415244204552526C
:10AB2F004F520043414C00494E4900454550000AE1
:10AB3F00414E54494352555348494E472044495377
:10AB4F0041424C4544002D2D2D0052414D004552A0
:10AB5F005200402823293D3D3D2053797374656D84
:10AB6F00203D3D3D3D3D3D3D3D3D3D3D3D3D00405D
:10AB7F00282329205345444543414C205820504C0D
:10AB8F00555300402823293D3D3D3D3D3D3D3D3D35
:10AB9F003D3D3D3D3D3D3D3D3D3D3D3D3D3D3D0013
:10ABAF00402823292D2D2D20536F667477617265F0
:10ABBF002056657273696F6E202D2D2D004028234E
:10ABCF0029563036205230322E3500402823292D79
:10ABDF002D2D20436F6D70696C6174696F6E204409
:10ABEF00617465202D2D2D0040282329417072207E
:10ABFF003235203230303600402823292D2D2D209C
:10AC0F00436F6D70696C6174696F6E2054696D6507
:10AC1F00202D2D2D004028232931353A34363A3254
:10AC2F003200402823292D2D2D20436F6D70696C24
:10AC3F0065722056657273696F6E202D2D2D004041
:10AC4F00282329372E303100402823292D2D2D2060
:10AC5F004D656D6F7279204D6F64656C202D2D2DB4
:10AC6F002D2D2D2D00402823293200402823292D5A
:10AC7F002D2D2D2D2D2D2D2D2D2D2D2D2D2D2D2DF5
:10AC8F002D2D2D2D2D2D2D005630360052322E35D7
:09AC9F00002020200000FF55AA4E
:10B98600780A7C007D017BFF7AAC79A07E007F047B
:10B99600122CA1E4900008F0E4900009F090000950
:10B9A600E0FFC394035055740A2FF582E43400F582
:10B9B60083742DF09000D37401F0A37400F0A37487
:10B9C6000AF07B017A01792912D036900009E02429
:10B9D6000AF582E43400F5837420F012E05D9001EC
:10B9E600B8E4F0A37433F012002E9001B8E07002B0
:10B9F600A3E070F6900009E004F080A1900008E052
:10BA060004F0E0C3940140909000D374FFF0A37457
:10BA1600ACF0A37497F07B017A01792912D0361223
:10BA2600E05D9001B8E4F0A37465F012002E900179
:10BA3600B8E07002A3E070F69000D374FFF0A37430
:10BA4600ACF0A3749BF07B017A01792912D03612EF
:10BA5600E05D9001B8E4F0A37465F012002E900149
:10BA6600B8E07002A3E070F69000D374FFF0A37400
:10BA7600ABF0A3741FF07B017A01792912D036222C
:10703100E4900006F0A3F0C2037825762008F678E4
:1070410029763008F67839764008F67827765008A0
:10705100F6782D766008F67823767008F6782F7624
:107061008008F67835769008F6783176A008F678BB
:107071002B76B008F6783776C008F643B74012D9B8
:10708100B512E020D2AF12BB6512E03712BA8612F8
:10709100BF9712CF5A12B51812B98612BF9712E0D4
:1070A1002812BF97E4900005F0900005E0FFD3940B
:1070B100054006EFD39402500B12A105900005E0A4
:1070C10004F080E57F0612C89CEF64017003027131
:1070D1006E7F0612C89CEF6402700302716E7F021C
:1070E10012C89CEF6401700302716E7F0212C89C8A
:1070F100EF640260787F0112C89CEF6401606E7FCB
:107101000112C89CEF640260647F0312C89CEF64A3
:1071110001605A7F0312C89CEF640260507F041221
:10712100C89CEF640160467F0412C89CEF64026052
:107131003C7F0512C89CEF640160327F0512C89C38
:0A714100EF64026028E4FF12C89C0E
:10714B00EF6401601EE4FF12C89CEF640260147FC1
:10715B000712C89CEF6401600A7F0712C89CEF649A
:10716B000270647B017A01798E7D0412CD04400399
:10717B000274A6C2057F3F12DBD0C2057F0312DC6F
:10718B0010E4900120F090018FF09001C7F0900176
:10719B009BF09001C6F090013CF07F0512DF277F3A
:1071AB000412DF277F0312DF277F0212DF277F0105
:1071BB0012DF27E4FF12DF277F0512D8FE7BFF7A51
:1071CB00AB792312860C227F0712C92FEF64016063
:1071DB00087F0712C92FBF0204D2108002C21020F1
:1071EB00100302730F9000D374FFF0A374ABF0A3E2
:1071FB007432F07B017A01792912D03612E05D905E
:10720B0001B87401F0A3742DF012002E9001B8E0B8
:10721B007002A3E070F6E4900005F0900005E0FF2B
:10722B00D394054006EFD39402500B12A1059000A6
:10723B0005E004F080E57F0612C89CEF6401600D49
:10724B007F0612C89CEF6402600302730F7F021269
:10725B00C89CEF6401700302730F7F0212C89CEF8E
:0D726B006402700302730F7F0112C89CEFD4
:107278006401600D7F0112C89CEF64026003027311
:107288000F7F0312C89CEF6401600A7F0312C89C39
:10729800EF640270727F0412C89CEF640160687F1B
:1072A8000412C89CEF6402605E7F0512C89CEF64FC
:1072B80001600A7F0512C89CEF6402704A9000D3EF
:1072C80074FFF0A374ABF0A37436F07B017A0179F4
:1072D8002912D03612E05D9001B8E4F0A37465F08D
:1072E80012002E9001B8E07002A3E070F69000D36F
:1072F80074FFF0A374ABF0A3743AF07B017A0179C0
:107308002912D036123F0E7B017A01798E125283F0
:10731800900006E0FEA3E0FFC39405EE648094802D
:10732800502FEF94FBEE6480947F402520B30DE04E
:1073380004F07006900006E004F0800E900007E06C
:1073480024FFF0900006E034FFF07F5B12DFF78047
:10735800BFD3900007E09400900006E0648094801A
:10736800407CD2047F4012DBF0E4900006F0A3F0EA
:1073780012E05D9001B87401F0A374F5F012002ECC
:067388009001B8E0700264
:10738E00A3E070F6900006E0FEA3E0FFC39405EEC6
:10739E0064809480502FEF94FBEE6480947F4025A0
:1073AE0030B30DE004F07006900006E004F0800E9D
:1073BE00900007E024FFF0900006E034FFF07F5BC2
:1073CE0012DFF780BFD3900007E09400900006E034
:1073DE00648094804002D20320036EC2057F3F1268
:1073EE00DBD0C2057F0312DC10E4900120F0900187
:1073FE008FF09001C7F090019BF09001C6F09001C4
:10740E003CF07F0512DF277F0412DF277F0312DF98
:10741E00277F0212DF277F0112DF27E4FF12DF270B
:10742E007F0712D8FE7BFF7AAB793E12860C3010A6
:10743E000D7B017A01798E7D0312CD04800B7B01C9
:10744E007A01798E7D0412CD0490018EE0FF6404E2
:10745E00601CEF640360179000D374FFF0A374AB4D
:10746E00F0A37455F07B017A01792912D03612E01F
:10747E005D9001B8E4F0A37465F012002E9001B88F
:10748E00E07002A3E070F67B017A01798E12E04B78
:09749E00D288D28AD2A8D2AA2217
:10CAE600E47812F6E47810F608F67813F608F67885
:10CAF60013E6FE08E6FFC3EE6480948450247812A1
:10CB0600E690ACA493FD7810E6FA08E68A832FF542
:10CB160082E5833EF583EDF0781406E6187001068B
:10CB260080CDE47810F608F67813F608F67813E662
:10CB3600FE08E6FFC3EE6480948450297810E6FC74
:10CB460008E68C832FF582E5833EF583E0FF08E651
:10CB560090ACA493FEEF6E6002C322781406E6182A
:10CB660070010680C8781206E66404600302CAEA09
:02CB7600D322C8
:10977C0078147900740090000075A22012FFF07527
:10978C00A200F50AB41505E4F58E8006758F0175F7
:10979C008E2D7800740008F6B8FFFB780008E6B44C
:1097AC000041B8FFF8780074FF08F6B8FFFB7800AA
:1097BC0008E6B4FF2EB8FFF87800745508F6B8FF29
:1097CC00FB780008E6B4551BB8FFF8780074AA08BB
:1097DC00F6B8FFFB780008E6B4AA08B8FFF875F0F5
:1097EC0001800375F000787FE4F6D8FDE5F0F5080C
:1097FC0012CAE6E433F50912D0A2127031E5086002
:10980C0004E509706B7B017A01797712DD00900019
:10981C00D374FFF0A374ABF0A37459F07B017A01FD
:10982C00792912D03612E05D9001B8E4F0A374658A
:10983C00F012002E9001B8E07002A3E070F69000D8
:10984C00D374FFF0A374ABF0A3745DF07B017A01C9
:10985C00792912D03612E05D9001B8E4F0A374655A
:10986C00F012002E9001B8E07002A3E060A080F42A
:10987C0012001690027EE054FDF09001B7E07018D3
:10988C0012CFC97B017A01792912C9C27B017A01F5
:05989C00797712C9C23A
:1098A10012DF8390027EE054FBF09001B6E0700677
:1098B100129F3C12DF909001BAE0701A900188E08B
:1098C100701190018EE0FF64046008EF640360038F
:1098D10012DA2812DF9D90027EE054F7F09001B574
:1098E100E0706D12A10512001E12DDC612DDDC1240
:1098F100DDF290018EE064017056900188E0B409B8
:1099010000504D90990BF828287302994402993020
:1099110002992602993A02992B02993F029949022A
:10992100993502994E128BC4802612DD8080211256
:109931005B7F801C125B7F801712AFB3801212DD38
:109941004E800D12003680081233BF800312497811
:1099510090027EE054EFF090018EE024FC6012044E
:10996100600302987F7B017A01798E1282B7029897
:0E9971007F7B017A01798E12E05102987F22ED
:08E01800434F4E0043414C0050
:10CD04009000D0EBF0A3EAF0A3E9F0A3EDF0C205A4
:10CD14007F3F12DBD0C2057F0312DC10E4900120B8
:10CD2400F090018FF09001C7F090019BF09001C644
:10CD3400F090013CF07F0512DF277F0412DF277F8C
:10CD44000312DF277F0212DF277F0112DF27E4FFB0
:10CD540012DF279000D0E0FBA3E0FAA3E0F9122C45
:10CD6400C7FF64046014EFB403079000D3E0B40475
:0CCD7400099000D3E0122D40D322C3220E
:06E04B007D0112CD04224C
:1082B700900005EBF0A3EAF0A3E9F090014DE0246C
:1082C700CDFF90014CE03400FE900154E0FCA3E0A8
:1082D700FD2FFFEC3EFEC3900145E09FEE6480F862
:1082E700900144E064809850030283F390014DE0CD
:1082F700245AFF90014CE03400CF2DCF3CFEC390B1
:10830700015BE09FEE6480F890015AE0648098502A
:10831700030283F3E4FFFE12CDF8EF246EFFE43E81
:10832700FE900144E0FCA3E0FDC39FEE6480F8ECFF
:1083370064809850030283F3900147E0246EFF9016
:108347000146E03400FEC3ED9FEE6480F8EC6480E4
:108357009850030283F3900154E0FEA3E0FF9001DD
:108367004DE02FFF90014CE03EFEC3900149E09F96
:10837700EE6480F8900148E0648098406FE4FFFE67
:1083870012CDF890015AE0FCA3E0FDC39FEE648094
:10839700F8EC6480984055900146E0FEA3E0FFEDBD
:1083A7009FEE6480F8EC6480984041E4FDFCFFFE9A
:1083B7001266F6C006C007E4FFFE12CDF8D005D05E
:1083C70004C3ED9FEE6480F8EC648098401EE4FDE2
:1083D700FCFFFE1266F6D3900147E09FEE6480F83B
:1083E700900146E064809850030284797F0312C8A5
:1083F7009CEF6401600D7F0312C89CEF6402600369
:1084070002860B7F0412C89CEF6401600D7F041283
:10841700C89CEF6402600302860B7F0512C89CEFBD
:108427006401600D7F0512C89CEF64026003028639
:108437000B9001887403F012BF97900005E0FBA32F
:10844700E0FAA3E0F97401122D4090017DE0B4FF3A
:10845700097B017A01797712DD009000D374FFF070
:10846700A374E0F0A37418F07B017A01792912D084
:108477003622128925400302851720100302860B36
:108487007F0112C89CEF6401600D7F0112C89CEF49
:108497006402600302860B7F0212C89CEF640160CE
:1084A7000D7F0212C89CEF6402600302860B7F06F1
:1084B70012C89CEF6401600D7F0612C89CEF64022E
:1084C700600302860B12D7B2900005E0FBA3E0FA27
:1084D700A3E0F97401122D40D20F90018804F01225
:1084E700BF9790018A74FFF090017DE0B4FF097B8C
:1084F700017A01797712DD009000D374FFF0A3743D
:10850700E0F0A3741CF07B017A01792912D036229E
:108517007DFF7F0712DAEC7F0712C92FEF64046033
:108527000302860B7F0112C89CEF64017003028669
:108537000B7F0112C89CEF6402700302860B7F0257
:1085470012C89CEF6401700302860B7F0212C89C5D
:10855700EF6402700302860B7F0312C89CEF64016D
:10856700700302860B7F0312C89CEF64027003023C
:10857700860B7F0412C89CEF6401700302860B7F91
:108587000412C89CEF6402607B7F0512C89CEF64ED
:108597000160717F0512C89CEF640260677F061255
:1085A700C89CEF6401605D7F0612C89CEF6402609F
:1085B70053E4FF12C89CEF64016049E4FF12C89CB2
:1085C700EF6402603F7F0712C89CEF640160357F4C
:1085D7000712C89CEF6402602B900005E0FBA3E044
:1085E700FAA3E0F97401122D4012BF977F0712DF3B
:1085F7002790017DE0B4FF097B017A01797712DDCD
:058607000012DEE32279
:06E051007404122D4022B0
:06E05700E4FF12DFF722D6
:10DD1A00C2B512E057D2B412E057D2B512E057C2D8
:0ADD2A00B412E057C2B512E0572210
:10DD9800C2B412E057D2B512E057D2B412E057C25B
:07DDA800B512E057C2B422DE
:05D4AB009000F7EFF016
:10D4B000E4A3F09000F7E0FF30E704D2B48002C2AA
:10D4C000B4EF25E09000F7F012E057D2B512E05724
:10D4D000C2B512E0579000F8E004F0E0C3940840B1
:10D4E000D2D2B412E057D2B512E05730B408C2B568
:0DD4F00012E0577F0122C2B512E0577F0005
:01D4FD00220C
:05D3AC009000F7EFF016
:10D3B100E49000F9F0D2B412E057E49000F8F0D212
:10D3C100B512E0579000F9E0FF25E0F030B403E03A
:10D3D10004F0C2B512E0579000F8E004F0E0C39405
:10D3E1000840DC9000F7E06004D2B48002C2B412BD
:10D3F100E057D2B512E057C2B512E0579000F9E0FC
:01D40100FF2B
:01D402002207
:07E0370012DD1A12DD982230
:10CB78009000F0EFF0A3EDF0A3EBF0A3EAF0A3E947
:01CB8800F0BC
:10CB8900C20512DD1A9000F0E0FF12D4ABBF01021A
:10CB9900D2059000F1E0FF12D4ABBF0102D205E447
:10CBA9009000F6F09000F5E0FFA3E0FEC39F502649
:10CBB9009000F2E0FBA3E0FAA3E0F98E827583000E
:10CBC900122CE0FF12D4ABBF0104D20580089000FB
:10CBD900F6E004F080CE12DD98E49000F6F07F5B79
:10CBE90012DFF79000F6E004F0E0C3945440EF3010
:07CBF90005037F01227F000C
:01CC00002211
:10C628009000F0EFF0A3EDF0A3EBF0A3EAF0A3E99C
:01C63800F011
:10C63900C20512DD1A9000F0E0FF12D4ABBF01026F
:10C64900D2059000F1E0FF12D4ABBF0102D205126E
:10C65900DD1A9000F0E04401FF12D4ABBF0102D211
:10C66900059000F5E014F0E4A3F09000F5E0FFA3D5
:10C67900E0C39F5025E4FF12D3AC9000F2E0FBA386
:10C68900E0FAA3E0F99000F6E0F582758300EF1275
:10C699002D529000F6E004F080D07FFF12D3AC90C9
:10C6A90000F2E0FBA3E0FAA3E0F9A3E0F5827583C9
:10C6B90000EF122D5212DD983005037F01227F0011
:01C6C900224E
:10D9B500E49001B5F09001B7F0A3F0A3F09001B6A3
:10D9C500F09001BAF0A3F0A3F09001BEF09001C071
:10D9D500F09001BFF09001C1F09001B47409F07F9F
:0AD9E5000112D176500312DD342246
:0400160012DB1422C3
:10B299009001B4E0600514F002B3D39001B7E06007
:10B2A9000214F09001B8E07002A3E0600E9001B9B9
:10B2B900E024FFF09001B8E034FFF09001BAE060BB
:10B2C9000214F09001BBE0600514F002B36590012F
:10B2D90095E0F4600302B36512A1057F0312C89CCF
:10B2E900EF640460087F0412C89CBF0418C2057F7C
:10B2F9000212DBD0E49001C7F0C2057F0112DBD056
:10B30900E490019BF07F0512C89CEF640460087FFC
:10B319000612C89CBF0418C2057F0412DBD0E49052
:10B32900013CF0C2057F0812DBD0E49001C6F07F32
:10B339000112C89CEF640460087F0212C89CBF0414
:10B3490018C2057F1012DBD0E4900120F0C2057FFE
:10B359002012DBD0E490018FF012DFAA9001BCE04B
:10B36900600214F09001BDE0600414F08036900191
:10B379003BE06030C2057F1012DBD0E4900120F081
:10B38900C2057F2012DBD0E490018FF0C2057F084F
:10B3990012DBD0E49001C6F0C2057F0412DBD0E4D1
:10B3A90090013CF09001BEE0600214F09001C0E011
:10B3B900600214F09001BFE0600214F09001C1E056
:10B3C900600214F09001B47409F09001B5E06002D4
:0BB3D90014F09001B6E0600214F022B6
:0D001E0012E05D9001B5740BF012002E226F
:0DDF830012E05D9001B7741AF012002E221A
:0DDF900012E05D9001B6740BF012002E221D
:0DDF9D0012E05D9001BA7433F012002E22E4
:0DDFAA0012E05D9001BB741AF012002E22EF
:0DDFB70012E05D9001BC7465F012002E2296
:0DDFC40012E05D9001BD74C9F012002E2224
:10DE7000900059EFF012E05D900059E09001BEF083
:04DE800012002E223C
:10DE8400900059EFF012E05D900059E09001C0F06D
:04DE940012002E2228
:10DE9800900059EFF012E05D900059E09001BFF05A
:04DEA80012002E2214
:0DDFD10012E05D9001C174D1F012002E220B
:0BDFF700E4FEEEC39F5004000E80F714
:01E0020022FB
:05D17600900008EFF03D
:10D17B00A3122FEE0000FFFF900009E0FCA3E0FDDF
:10D18B00A3E0FEA3E0FFE47B06FAF9F8122E54901D
:10D19B000009122FE2900009E0FCA3E0FDA3E0FEE2
:10D1AB00A3E0FFE47B207A4EF9F8122EDF90000902
:10D1BB00122FE2900008E0FFE4FCFDFEA3E0F8A3D1
:10D1CB00E0F9A3E0FAA3E0FBC3122F7F5002C322C6
:01D1DB00D380
:01D1DC002230
:03000B0002001AD6
:01001A0032B3
:03001B00020032AE
:01003200329B
:03002B00020006CA
:05000600C2CEC2CF32A2
:10DDAF00454550524F4D204552524F52000602A04A
:07DDBF00A2A4A6A8AAACAEC5
:10BC4100E49000EDF0A3F0A3F09000DCF0E49000AC
:10BC5100DBF09000DBE0FFC39410506FEFC454F0B1
:10BC6100FE9000EDE0FFC0079000DCE090DDBE93A8
:10BC7100FFAD067B017A0079DD9000F57410F012BA
:10BC8100C628D0E04F9000EDF0E4FF9000DCE0FE2C
:10BC9100B4030C9000DBE0B40F05EF640E6024EEFA
:10BCA100C39404501974DD2FF582E43400F583E068
:10BCB100FD9000EFE02DF09000EEE03400F00FEF8A
:10BCC100B410C89000DBE004F080879000DCE00451
:10BCD100F0E0C39404500302BC4E9000EDE0FEC0BE
:10BCE100067B017A0079EE9000F57402F07DFE7F0B
:10BCF100A612CB78D0E04F9000EDF0E0FEC0067BBD
:10BD0100017A0079EE9000F57402F07DFE7FAE12AB
:0ABD1100CB78D0E04FFF9000EDF07A
:01BD1B002205
:103F0E00E490001AF0900008F0900008E0FFC394CF
:103F1E00105014740A2FF582E43400F583E4F09007
:103F2E000008E004F080E2E4900009F0E49000085C
:103F3E00F0900008E0FFC394105038EFC454F0FF27
:103F4E0090001BF0FD90001AE0FEC006900009E004
:103F5E0090DDBE93FF7B017A00790A9000F5741014
:103F6E00F012CB78D0E04F90001AF0900008E004E9
:103F7E00F080BE900009E004F0E0C3940840AD90DC
:103F8E00001AE064017003024972E490001CF0A371
:103F9E00F090001AE0FEC0067B017A00791C9000BA
:103FAE00F57402F0E4FD7FA012CB78D0E04F9000C4
:103FBE001AF0E0FEC0067B017A00791C9000F574C1
:103FCE0002F0E4FD7FA812CB78D0E04F90001AF0FB
:103FDE0090001C7404F0A3E4F090001AE0FEC006FA
:103FEE007B017A00791C9000F57402F0FD7FA0121F
:103FFE00CB78D0E04F90001AF0E0FEC0067B017A3D
:10400E0000791C9000F57402F0FD7FA812CB78D0D9
:10401E00E04F90001AF090001C7402F0A37426F08A
:10402E0090001AE0FEC0067B017A00791C9000F524
:10403E007402F07D047FA012CB78D0E04F90001A6E
:10404E00F0E0FEC0067B017A00791C9000F5740248
:10405E00F07D047FA812CB78D0E04F90001AF0E4E8
:10406E0090001CF0A3F090001AE0FEC0067B017ACF
:10407E0000791C9000F57402F07D067FA012CB78BB
:10408E00D0E04F90001AF0E0FEC0067B017A007976
:10409E001C9000F57402F07D067FA812CB78D0E05C
:1040AE004F90001AF090001C7401F0A37455F0901C
:1040BE00001AE0FEC0067B017A00791C9000F574B0
:1040CE0002F07D087FA012CB78D0E04F90001AF05E
:1040DE00E0FEC0067B017A00791C9000F57402F0B8
:1040EE007D087FA812CB78D0E04F90001AF0900098
:1040FE001C7402F0A374AAF090001AE0FEC0067BB6
:10410E00017A00791C9000F57402F07D0A7FA012EE
:10411E00CB78D0E04F90001AF0E0FEC0067B017A1B
:10412E0000791C9000F57402F07D0A7FA812CB78FE
:10413E00D0E04F90001AF090001C7404F0A3E4F04D
:10414E0090001AE0FEC0067B017A00791C9000F503
:10415E007402F07D0C7FA012CB78D0E04F90001A45
:10416E00F0E0FEC0067B017A00791C9000F5740227
:10417E00F07D0C7FA812CB78D0E04F90001AF0E4BF
:10418E0090001CF0A3F090001AE0FEC0067B017AAE
:10419E0000791C9000F57402F07D0E7FA012CB7892
:1041AE00D0E04F90001AF0E0FEC0067B017A007955
:1041BE001C9000F57402F07D0E7FA812CB78D0E033
:1041CE004F90001AF090001C7404F0A3E4F09000DD
:1041DE001AE0FEC0067B017A00791C9000F574028D
:1041EE00F07D107FA012CB78D0E04F90001AF0E057
:1041FE00FEC0067B017A00791C9000F57402F07DFA
:10420E00107FA812CB78D0E04F90001AF0E4900007
:10421E001CF0A3F090001AE0FEC0067B017A007934
:10422E001C9000F57402F07D127FA012CB78D0E0C6
:10423E004F90001AF0E0FEC0067B017A00791C90C8
:10424E0000F57402F07D127FA812CB78D0E04F906B
:10425E00001AF090001C7402F0A3E4F090001AE033
:10426E00FEC0067B017A00791C9000F57402F07D89
:10427E00147FA012CB78D0E04F90001AF0E0FEC071
:10428E00067B017A00791C9000F57402F07D147F94
:10429E00A812CB78D0E04F90001AF090001C740456
:1042AE00F0A3E4F090001AE0FEC0067B017A0079DC
:1042BE001C9000F57402F07D167FA012CB78D0E032
:1042CE004F90001AF0E0FEC0067B017A00791C9038
:1042DE0000F57402F07D167FA812CB78D0E04F90D7
:1042EE00001AF0E490001CF0A3F090001AE0FEC05B
:1042FE00067B017A00791C9000F57402F0E4FD7FD4
:10430E00A212CB78D0E04F90001AF0E0FEC0067BF0
:10431E00017A00791C9000F57402F0E4FD7FAA1278
:10432E00CB78D0E04F90001AF090001C7401F0A3EF
:10433E00745EF090001AE0FEC0067B017A00791CD4
:10434E009000F57402F0FD7FA212CB78D0E04F9072
:10435E00001AF0E0FEC0067B017A00791C9000F591
:10436E007402F0FD7FAA12CB78D0E04F90001AF0C5
:10437E0090001CE4F0A37478F090001AE0FEC006E2
:10438E007B017A00791C9000F57402F07D047FA207
:10439E0012CB78D0E04F90001AF0E0FEC0067B0101
:1043AE007A00791C9000F57402F07D047FAA12CB7E
:1043BE0078D0E04F90001AF090001CE4F0A3744106
:1043CE00F090001AE0FEC0067B017A00791C900086
:1043DE00F57402F07D067FA212CB78D0E04F9000EC
:1043EE001AF0E0FEC0067B017A00791C9000F5748D
:1043FE0002F07D067FAA12CB78D0E04F90001AF023
:10440E0090001CE4F0A3744BF090001AE0FEC0067E
:10441E007B017A00791C9000F57402F07D087FA272
:10442E0012CB78D0E04F90001AF0E0FEC0067B0170
:10443E007A00791C9000F57402F07D087FAA12CBE9
:10444E0078D0E04F90001AF090001CE4F0A3740AAC
:10445E00F090001AE0FEC0067B017A00791C9000F5
:10446E00F57402F07D0A7FA212CB78D0E04F900057
:10447E001AF0E0FEC0067B017A00791C9000F574FC
:10448E0002F07D0A7FAA12CB78D0E04F90001AF08E
:10449E0090001CE4F0A37432F090001AE0FEC00607
:1044AE007B017A00791C9000F57402F07D0C7FA2DE
:1044BE0012CB78D0E04F90001AF0E0FEC0067B01E0
:1044CE007A00791C9000F57402F07D0C7FAA12CB55
:1044DE0078D0E04F90001AF090001CE4F0A37432F4
:1044EE00F090001AE0FEC0067B017A00791C900065
:1044FE00F57402F07D0E7FA212CB78D0E04F9000C3
:10450E001AF0E0FEC0067B017A00791C9000F5746B
:10451E0002F07D0E7FAA12CB78D0E04F90001AF0F9
:10452E0090001CE4F0A374BEF090001AE0FEC006EA
:10453E007B017A00791C9000F57402F07D107FA249
:10454E0012CB78D0E04F90001AF0E0FEC0067B014F
:10455E007A00791C9000F57402F07D107FAA12CBC0
:10456E0078D0E04F90001AF090001CE4F0A3740F86
:10457E00F090001AE0FEC0067B017A00791C9000D4
:10458E00F57402F07D127FA212CB78D0E04F90002E
:10459E001AF0E0FEC0067B017A00791C9000F574DB
:1045AE0002F07D127FAA12CB78D0E04F90001AF065
:1045BE0090001CE4F0A374B4F090001AE0FEC00664
:1045CE007B017A00791C9000F57402F07D147FA2B5
:1045DE0012CB78D0E04F90001AF0E0FEC0067B01BF
:1045EE007A00791C9000F57402F07D147FAA12CB2C
:1045FE0078D0E04F90001AF090001CE4F0A3742DD8
:10460E00F090001AE0FEC0067B017A00791C900043
:10461E00F57402F07D167FA212CB78D0E04F900099
:10462E001AF0E0FEC0067B017A00791C9000F5744A
:10463E0002F07D167FAA12CB78D0E04F90001AF0D0
:10464E0090001CE4F0A374A3F090001AE0FEC006E4
:10465E007B017A00791C9000F57402F07D187FA220
:10466E0012CB78D0E04F90001AF0E0FEC0067B012E
:10467E007A00791C9000F57402F07D187FAA12CB97
:10468E0078D0E04F90001AF090001CE4F0A374690B
:10469E00F090001AE0FEC0067B017A00791C9000B3
:1046AE00F57402F07D1A7FA212CB78D0E04F900005
:1046BE001AF0E0FEC0067B017A00791C9000F574BA
:1046CE0002F07D1A7FAA12CB78D0E04F90001AF03C
:1046DE0090001C74FFF0A374E2F090001AE0FEC08C
:1046EE00067B017A00791C9000F57402F07D1C7F28
:1046FE00A212CB78D0E04F90001AF0E0FEC0067BFD
:10470E00017A00791C9000F57402F07D1C7FAA12CC
:10471E00CB78D0E04F90001AF0E490001CF0A3F09C
:10472E0090001AE0FEC0067B017A00791C9000F51D
:10473E007402F07D1E7FA212CB78D0E04F90001A4B
:10474E00F0E0FEC0067B017A00791C9000F5740241
:10475E00F07D1E7FAA12CB78D0E04F90001AF09019
:10476E00001CE4F0A3745AF090001AE0FEC0067B21
:10477E00017A00791C9000F57402F07D207FA21260
:10478E00CB78D0E04F90001AF0E0FEC0067B017AA5
:10479E0000791C9000F57402F07D207FAA12CB7870
:1047AE00D0E04F90001AF090001CE4F0A37478F063
:1047BE0090001AE0FEC0067B017A00791C9000F58D
:1047CE007402F07D227FA212CB78D0E04F90001AB7
:1047DE00F0E0FEC0067B017A00791C9000F57402B1
:1047EE00F07D227FAA12CB78D0E04F90001AF09085
:1047FE00001CE4F0A37464F090001AE0FEC0067B87
:10480E00017A00791C9000F57402F07D247FA212CB
:10481E00CB78D0E04F90001AF0E0FEC0067B017A14
:10482E0000791C9000F57402F07D247FAA12CB78DB
:10483E00D0E04F90001AF090001CE4F0A374B4F096
:10484E0090001AE0FEC0067B017A00791C9000F5FC
:10485E007402F07D267FA212CB78D0E04F90001A22
:10486E00F0E0FEC0067B017A00791C9000F5740220
:10487E00F07D267FAA12CB78D0E04F90001AF090F0
:10488E00001C74FFF0A374A6F090001AE0FEC006A0
:10489E007B017A00791C9000F57402F07D287FA2CE
:1048AE0012CB78D0E04F90001AF0E0FEC0067B01EC
:1048BE007A00791C9000F57402F07D287FAA12CB45
:1048CE0078D0E04F90001AF0E490001CF0A3F09026
:1048DE00001AE0FEC0067B017A00791C9000F57488
:1048EE0002F07D2A7FA212CB78D0E04F90001AF012
:1048FE00E0FEC0067B017A00791C9000F57402F090
:10490E007D2A7FAA12CB78D0E04F90001AF090004B
:10491E001CE4F0A3745AF090001AE0FEC0067B016E
:10492E007A00791C9000F57402F07D2C7FA212CBD8
:10493E0078D0E04F90001AF0E0FEC0067B017A00BE
:10494E00791C9000F57402F07D2C7FAA12CB78D0E2
:10495E00E04F90001AF0E0FEC00612BC41D0E04FCE
:09496E0090001AF090001AE0FF1D
:01497700221D
:0B528300900008EBF0A3EAF0A3E9F0B4
:10528E00E490001EF0C204900020F0A3F0A3F0A35F
:10529E00F090000DF0E490000CF090000CE0FFC3D5
:1052AE00941040030253F9EFC454F0FF90001FF026
:1052BE00FD90001EE0FEC00690000DE090DDBE9356
:1052CE00FF7B017A00790E9000F57410F012C6285B
:1052DE00D0E04F90001EF0E490000BF090000BE039
:1052EE00FFC3941040030253F090000DE0FE6403E0
:1052FE006008EE640760030253A490000CE0640F94
:10530E0060030253A4EFD3940D50030253A4A3E001
:10531E006403704290000BE0FFB40E1F240EF58262
:10532E00E43400F583E0FF900024E4F0A3EFF0E016
:10533E00F8E4F0E8900024F00253E790000BE0242C
:10534E000EF582E43400F583E0FF900024E0F0A334
:10535E00E04FF00253E790000BE0FFB40E1E240E58
:10536E00F582E43400F583E0FF900026E4F0A3EF2D
:10537E00F0E0F8E4F0E8900026F0805D90000BE09D
:10538E00240EF582E43400F583E0FF900026E0F071
:10539E00A3E04FF0804390000DE0C39404501E90A4
:1053AE00000BE0240EF582E43400F583E0FF90005C
:1053BE0021E02FF0900020E03400F0801C90000BD4
:1053CE00E0240EF582E43400F583E0FF900023E044
:1053DE002FF0900022E03400F090000BE004F00279
:1053EE0052EA90000CE004F00252A890000DE00486
:1053FE00F0E0C3940850030252A390001EE0640133
:10540E007069900008E0FBA3E0FAA3E0F97D0412B6
:10541E00CD044003025B7EC2057F3F12DBD0C20586
:10542E007F0312DC10E4900120F090018FF09001C8
:10543E00C7F090019BF09001C6F090013CF07F0503
:10544E0012DF277F0412DF277F0312DF277F02126E
:10545E00DF277F0112DF27E4FF12DF277F0112D83B
:10546E00FE7BFF7ADD79AF12860C22900024E0FEDF
:10547E00A3E0FF900020E0FCA3E0FDB50734ECB5FF
:10548E000630900026E0FEA3E0FF900022E0FAA393
:10549E00E0FBB5071DEAB50619E4900028F0ED6BA8
:1054AE007002EC6A700302556CA37404F0D204020D
:1054BE00556C900024E0FEA3E0FF900020E0B506BE
:1054CE0013A3E0B5070EE4900028F0A37404F0D205
:1054DE000402556C900026E0FEA3E0FF900022E04F
:1054EE00B50612A3E0B5070D9000287404F0E4A3EE
:1054FE00F0D2048069900008E0FBA3E0FAA3E0F983
:10550E007D0412CD044003025B7EC2057F3F12DB99
:10551E00D0C2057F0312DC10E4900120F090018FC1
:10552E00F09001C7F090019BF09001C6F090013C05
:10553E00F07F0512DF277F0412DF277F0312DF279C
:10554E007F0212DF277F0112DF27E4FF12DF277FA2
:10555E000112D8FE7BFF7ADD79AF12860C22900005
:10556E001EE0FEC006900028E090DDBE93FF7B019A
:10557E007A01799C9000F57402F0E4FD12C628D0F1
:10558E00E04F90001EF0E0FEC006900028E090DD97
:10559E00BE93FF7B017A01799E9000F57402F0FDB7
:1055AE0012C628D0E04F90001EF0E0FEC00690001C
:1055BE0028E090DDBE93FF7B017A0179A09000F583
:1055CE007402F07D0412C628D0E04F90001EF0E069
:1055DE00FEC006900028E090DDBE93FF7B017A01AD
:1055EE0079A29000F57402F07D0612C628D0E04F25
:1055FE0090001EF0E0FEC006900028E090DDBE9305
:10560E00FF7B017A0179A49000F57402F07D0812F7
:10561E00C628D0E04F90001EF0E0FEC00690002895
:10562E00E090DDBE93FF7B017A0179A69000F574C0
:10563E0002F07D0A12C628D0E04F90001EF0E0FE68
:10564E00C006900028E090DDBE93FF7B017A0179C1
:10565E00A89000F57402F07D0C12C628D0E04F9091
:10566E00001EF0E0FEC006900028E090DDBE93FF25
:10567E007B017A0179AA9000F57402F07D0E12C6B4
:10568E0028D0E04F90001EF0E0FEC006900028E00B
:10569E0090DDBE93FF7B017A0179AC9000F5740228
:1056AE00F07D1012C628D0E04F90001EF0E0FEC034
:1056BE0006900028E090DDBE93FF7B017A0179AE63
:1056CE009000F57402F07D1212C628D0E04F9000C3
:1056DE001EF0E0FEC006900028E090DDBE93FF7B3A
:1056EE00017A0179B09000F57402F07D1412C6288B
:1056FE00D0E04F90001EF0E0FEC006900028E09033
:10570E00DDBE93FF7B017A0179B29000F57402F051
:10571E007D1612C628D0E04F90001EF0E0FEC006A7
:10572E00900028E090DDBF93FF7B017A01794490D1
:10573E0000F57402F0FD12C628D0E04F90001EF066
:10574E00E0FEC006900028E090DDBF93FF7B017A5B
:10575E000179429000F57402F0E4FD12C628D0E003
:10576E004F90001EF0E0FEC006900028E090DDBFD6
:10577E0093FF7B017A0179469000F57402F07D0467
:10578E0012C628D0E04F90001EF0E0FEC00690003A
:10579E0028E090DDBF93FF7B017A0179489000F5F8
:1057AE007402F07D0612C628D0E04F90001EF0E085
:1057BE00FEC006900028E090DDBF93FF7B017A01CA
:1057CE00794A9000F57402F07D0812C628D0E04F99
:1057DE0090001EF0E0FEC006900028E090DDBF9322
:1057EE00FF7B017A01794C9000F57402F07D0A126C
:1057FE00C628D0E04F90001EF0E0FEC006900028B4
:10580E00E090DDBF93FF7B017A01794E9000F57435
:10581E0002F07D0C12C628D0E04F90001EF0E0FE84
:10582E00C006900028E090DDBF93FF7B017A0179DE
:10583E00509000F57402F07D0E12C628D0E04F9005
:10584E00001EF0E0FEC006900028E090DDBF93FF42
:10585E007B017A0179529000F57402F07D1012C628
:10586E0028D0E04F90001EF0E0FEC006900028E029
:10587E0090DDBF93FF7B017A0179549000F574029D
:10588E00F07D1212C628D0E04F90001EF0E0FEC050
:10589E0006900028E090DDBF93FF7B017A017956D8
:1058AE009000F57402F07D1412C628D0E04F9000DF
:1058BE001EF0E0FEC006900028E090DDBF93FF7B57
:1058CE00017A0179589000F57402F07D1612C628FF
:1058DE00D0E04F90001EF0E0FEC006900028E09051
:1058EE00DDBF93FF7B017A01795A9000F57402F0C7
:1058FE007D1812C628D0E04F90001EF0E0FEC006C4
:10590E00900028E090DDBF93FF7B017A01795C90D7
:10591E0000F57402F07D1A12C628D0E04F90001EDA
:10592E00F0E0FEC006900028E090DDBF93FF7B0103
:10593E007A01795E9000F57402F07D1C12C628D0B3
:10594E00E04F90001EF0E0FEC006900028E090DDD3
:10595E00BF93FF7B017A0179609000F57402F07DB0
:10596E001E12C628D0E04F90001EF0E0FEC006903A
:10597E000028E090DDBF93FF7B017A0179629000F1
:10598E00F57402F07D2012C628D0E04F90001EF074
:10599E00E0FEC006900028E090DDBF93FF7B017A09
:1059AE000179649000F57402F07D2212C628D0E0D1
:1059BE004F90001EF0E0FEC006900028E090DDBF84
:1059CE0093FF7B017A0179669000F57402F07D24D5
:1059DE0012C628D0E04F90001EF0E0FEC0069000E8
:1059EE0028E090DDBF93FF7B017A0179689000F586
:1059FE007402F07D2612C628D0E04F90001EF0E013
:105A0E00FEC006900028E090DDBF93FF7B017A0177
:105A1E00796A9000F57402F07D2812C628D0E04F06
:105A2E0090001EF0E0FEC006900028E090DDBF93CF
:105A3E00FF7B017A01796C9000F57402F07D2A12D9
:105A4E00C628D0E04F90001EF0E0FEC00690002861
:105A5E00E090DDBF93FF7B017A01796E9000F574C3
:105A6E0002F07D2C12C628D0E04F90001EF02004CC
:105A7E0003025B11E490000CF0E490000BF0900038
:105A8E000BE0FFC39410506CEFC454F0FF90001F56
:105A9E00F0FD90001EE0FEC006900028E0FF900092
:105AAE000CE02F90DDBE93FF7B017A00790E900003
:105ABE00F57410F012C628D0E04F90001EF0E0FEF4
:105ACE00C006900029E0FF90000CE02F90DDBE9301
:105ADE00FF90001FE0FD7B017A00790E9000F574B7
:105AEE0010F012CB78D0E04F90001EF090000BE03B
:105AFE0004F0808A90000CE004F0E0C3940450039C
:105B0E00025A8790001EE064017065900008E0FB69
:105B1E00A3E0FAA3E0F97D0412CD045053C2057F31
:105B2E003F12DBD0C2057F0312DC10E4900120F09F
:105B3E0090018FF09001C7F090019BF09001C6F09C
:105B4E0090013CF07F0512DF277F0412DF277F03D1
:105B5E0012DF277F0212DF277F0112DF27E4FF12F9
:105B6E00DF277F0112D8FE7BFF7ADD79AF12860C1C
:015B7E002204
:0BD59F00900006EBF0A3EAF0A3E9F017
:10D5AA00EF25E0FFA3F0FD9000F57402F07FA212D0
:10D5BA00CB78BF01037F012212BC41BF01037F0167
:10D5CA0022900009E0FD900006E0FBA3E0FAA3E048
:10D5DA00F99000F57402F07FAA12CB78BF01037F9D
:04D5EA0001227F009B
:01D5EE00221A
:0BD5EF009000D7EBF0A3EAF0A3E9F0F6
:10D5FA00EF25E0FFA3F0FD9000F57402F07FA01282
:10D60A00CB78BF01037F012212BC41BF01037F0116
:10D61A00229000DAE0FD9000D7E0FBA3E0FAA3E055
:10D62A00F99000F57402F07FA812CB78BF01037F4E
:04D63A0001227F004A
:01D63E0022C9
:07E03E0075A61E75A6E12284
:08E02000E4F5D9D2AED2DE22F4
:04002E0043DB01228D
:04E05D0053DBFE2271
:10DB140090027E741EF0A37407F0A374D0F09002F8
:10DB24007A740DF0A37405F090027BE0F5EA90029C
:08DB34007AE0F5FA75DA4922E6
:10DD340090027C740DF0A37405F090027DE0F5EB85
:0ADD440090027CE0F5FB75DB49223C
:0300330002BDF318
:10BDF300C0E0C0F0C083C082C0D075D000C000C016
:0DBE030001C002C003C004C005C006C00796
:10BE100030D86390027FE07002A3E0601312E03E2E
:10BE2000900280E024FFF090027FE034FFF0801762
:10BE300090027EE0701112E03E90027E741EF0A32C
:10BE40007407F0A374D0F0900001E5EAF0900000D0
:10BE5000E5FAF090027AE0FEA3E0FF900001E02F07
:10BE6000F0900000E03EF0A3E0F5EA900000E0F57D
:10BE7000FAC2D843DA0130D93212B299900001E502
:10BE8000EBF0900000E5FBF090027CE0FEA3E0FF09
:10BE9000900001E02FF0900000E03EF0A3E0F5EB11
:0BBEA000900000E0F5FBC2D943DB017D
:10BEAB00D007D006D005D004D003D002D001D000EB
:0BBEBB00D0D0D082D083D0F0D0E03295
:10D23E00900008EFF0A3ECF0A3EDF0FFAE04EE3398
:10D24E0095E0FDFC7804122FA3C004C005C006C0F3
:10D25E0007900009E0FEA3E0FFEE3395E0FDFCF839
:10D26E00F9AA06AB07D007D006D005D004C3EF9BB2
:10D27E00FFEE9AFEED99FDEC98FC900008E025E09B
:0FD28E0025E0244DF582E43402F583122FE222CD
:0DB75C00900008ECF0A3EDF0900007EFF076
:10B7690025E025E0244DF582E43402F583C083C049
:10B7790082E0F8A3E0F9A3E0FAA3E0FB900008E077
:10B78900FEA3E0FFEE3395E0FDFCEB2FFFEA3EFE62
:10B79900E93DFDE83CFCD082D083122FE2900007FE
:10B7A900E0FB25E025E0244DF582E43402F583E051
:10B7B900FCA3E0FDA3E0FEA3E0FF7804122F909024
:10B7C900000AEEF0A3EFF0EB25E025E0244DF58229
:10B7D900E43402F583C083C082E0FCA3E0FDA3E06A
:10B7E900FEA3E0FFE47B07FAF9F8122E54D082D0C9
:10B7F90083122FE2900007E025E025E0244DF58231
:10B80900E43402F583C083C082E0FCA3E0FDA3E039
:10B81900FEA3E0FF7803122F90D082D083122FE28B
:10B82900900007E025E025E0244DF582E43402F597
:10B8390083C083C082E0F8A3E0F9A3E0FAA3E0FBA8
:10B84900900008E0FEA3E0FFEE3395E0FDFCEB2F4E
:10B85900FFEA3EFEE93DFDE83CFCD082D083122F91
:09B86900E290000AE0FEA3E0FFFA
:01B8720022B3
:10AE3000303E4141413E0000003100017F210000D1
:10AE40000000323149454321000000333649494171
:10AE50002200000034047F24140C000000354E5101
:10AE600051517200000036064949291E0000003782
:10AE700060504847400000003836494949360000D4
:10AE800000393C4A494930000000411F2444241F36
:10AE9000000000423649497F410000004322414101
:10AEA000413E000000443E41417F410000004541D9
:10AEB0004149497F00000046404048487F0000006B
:10AEC000472E4941413E000000487F0808087F00A6
:10AED00000004900417F41000000004A407E4101DE
:10AEE000020000004B412214087F0000004C0101C9
:10AEF00001017F0000004D7F2018207F0000004EE0
:10AF00007F0810207F0000004F3E4141413E00007D
:10AF10000050304848487F000000513D4241413ECA
:10AF200000000052314A4C487F0000005326494936
:10AF300049320000005440407F4040000000557EF0
:10AF40000101017E00000056700C030C700000002F
:10AF5000577C030C037C0000005863140814630042
:10AF600000005960100F10600000005A61514945FF
:10AF7000430000003F304845402000000020000012
:10AF80000000000000002B00081C08000000002D3D
:10AF900000080808000000005F017F210808000089
:10AFA000003D39454329080000002A22147F14225D
:03AFB0000000009E
:05D1DD009000EAEFF0F4
:10D1E20012DF5750089000EAE024D0FF229000EAB4
:10D1F200E0FF12DCE5501F9000EAE0FF12DF66500C
:10D202000D9000EAE0FF12DF169000EAEFF09000C6
:10D21200EAE024C9FF227F2475F009EFA42430F547
:10D2220082E5F034AEF583E493FE9000EAE0FDEE91
:0BD23200B50501220FEFB42BDF7F24B5
:01D23D0022CE
:109B7100502531642E2531642573000A0A5052455F
:109B81005353203220544F205341564520544845C9
:109B91002056414C55450A312B33202D20414C4C48
:109BA1004F57204D4F56454D454E540A342D535570
:109BB100424C4556454C2055500A362D5355424C82
:109BC1004556454C20444F574E0A352D5155495461
:109BD1000053455400454550524F4D204552524F78
:109BE1005200204F4B000A312B33202D20414C4C89
:109BF1004F57204D4F56454D454E540A322D534136
:109C010056452056414C55450A0A342D5355424C70
:109C11004556454C20555020362D5355424C4556FE
:109C2100454C20444F574E0A0A352D515549540091
:109C3100202020000A504C414345205448452045EE
:109C4100515549504D454E5420494E2054484520C8
:109C5100504F534954494F4E2053484F574E204976
:109C61004E20444953504C415920414E44205448C0
:109C7100454E20505245535320554E444552544170
:109C8100424C45000A43415554494F4E0A4D4F56E7
:109C9100454D454E5420574954484F555420534F34
:109CA1004654574152452052455354524943544911
:109CB1004F4E530A504C414345205448452045518D
:109CC1005549504D454E5420414E44205357495417
:109CD1004348204954204F46460025730A25730006
:109CE100434F4E46494755524154494F4E204552E4
:109CF100524F5200524F4F4D204D41582048454937
:109D010047485420544F4F2053484F525400524516
:109D110056494557204D4158204845494748542008
:109D2100414E44204445544543544F5220484549EF
:109D31004748540054484F524158204F5220554EE5
:109D41004445525441424C452048454947485420D6
:109D5100544F4F204849474800434F4E0043414C20
:019D61000001
:10D0A200E490018AF090018EF0900188F090017571
:10D0B200F0900176F090013BF0D20F9001C4E05461
:10D0C200FEF054FDF054FBF054F7F054EFF054DF4F
:10D0D200F054BFF0547FF0A3E054FEF054FBF05440
:10D0E200F7F0E49001C7F090019BF0900120F090DE
:10D0F200018FF09001C6F090013CF090013EF0905B
:0BD102000192F0900196F012D7B222CB
:10D35400D20F900188E090013DF0900188EFF01227
:10D36400BF97C2057F3F12DBD0C2057F0312DC10DA
:10D37400E4900120F090018FF09001C7F090019BA0
:10D38400F09001C6F090013CF07F0512DF277F0486
:10D3940012DF277F0312DF277F0212DF277F0112AC
:08D3A400DF27E4FF12DF27225E
:10DF4700D20F900188E0900141F0900188EFF02214
:09E00F00900141E0900188F0222B
:10DD8000300F08C20F12C13312DFB79001BCE07030
:08DD90000612C41D12E00F226F
:108BC400200F03028C8712DA90EF7003028E37C2F3
:108BD400A8C2AAC20F90013DE06401600812DF75CB
:108BE4007F0412DF4790018AE070787B019000D304
:108BF40004F0A37400F0A37406F0A3EBF0A37400D4
:108C0400F0A37407F0A3EBF0A37400F0A37408F0CE
:108C14007A00790512C0669000EB74FFF0A3749B90
:108C2400F0A37471F0900005E02401FEE433900099
:108C3400EEF0A3CEF0900006E02401FEE4339000B1
:108C4400F0F0A3CEF0A374FFF0A3749BF0A3747CA4
:108C5400F07B017A007908126C137B017A007908A1
:108C6400127BE5E490018AF07F0312D10D7DFF7F32
:108C74000212DAEC7F0112D10D7F0312DEBF7F05F1
:108C840012DEBF7F0312C89CBF010B12DC307F04CD
:108C940012DF47028D1B7F0512C89CBF010A12DD3B
:108CA400687F0412DF47806F7F0412C89CEF640161
:108CB400706512DF377F0412DF4712E03050137DF6
:108CC400FF7F0412DAECE4FF12D10D7F0512D10DFF
:108CD4008045C2057F3F12DBD0C2057F0312DC1042
:108CE400E4900120F090018FF09001C7F090019B77
:108CF400F09001C6F090013CF07F0512DF277F045D
:108D040012DF277F0312DF277F0212DF277F011282
:108D1400DF27E4FF12DF2712E0304003028DC67F15
:108D24000612C89CEF6401600A7F0612C89CEF64B7
:108D34000270397F0112C89CEF640160087F011240
:108D4400C89CBF02277F0112D3547F0312DF057F23
:108D54000512DF059000D774FFF0A3749BF0A37491
:108D6400D2F07B017A01792912CA54227F0212C8F7
:108D74009CEF64016003028E3712C76CBF011F7B36
:108D8400017A01798E7D0412CD044003028E377F6F
:108D94000112D8FE7BFF7A9B79D612860C229000B2
:108DA400D774FFF0A3749BF0A374E3F07B017A0102
:108DB400792912CA547BFF7A9B79E7127BE512D892
:108DC4003E227F0312D10D7DFF7F0212DAEC7F0178
:108DD40012D10D7F0112C89CEF6401600A7F011259
:108DE400C89CEF6402704C7F0212C89CEF6401605F
:108DF4000A7F0212C89CEF640270387F0612C89C76
:108E0400EF640160087F0612C89CBF0226E4FF12CB
:108E1400D3549000D374FFF0A3749CF0A37431F086
:108E24007B017A01792912D0367F0312DF057F0591
:038E340012DF0545
:018E37002218
:105B7F00300F2A12DA90EF70030261FDC20FC2A834
:105B8F00C2AA900188E0B4010B7BFF7A9C79351291
:105B9F007BE580097BFF7A9C7985127BE57F071275
:105BAF00C92FEF64016003025CD39001C4E0FFC30F
:105BBF001320E003025C807F0112C89CEF64017028
:105BCF0003025C807F0112C89CEF64027003025CC9
:105BDF00807F0212C89CEF64017003025C807F0219
:105BEF0012C89CEF64027003025C807F0312C89C92
:105BFF00EF6401607C7F0312C89CEF640260727FC8
:105C0F000412C89CEF640160687F0412C89CEF64A3
:105C1F0002605E7F0512C89CEF640160547F05121D
:105C2F00C89CEF6402604A7F0612C89CEF64016053
:105C3F00407F0612C89CEF64026036E4FF12C89CD6
:105C4F00EF6401602CE4FF12C89CEF640260227FB6
:105C5F000712C89CEF640160187F0712C89CEF649D
:105C6F0002600E9001C4E054FDF07F0712DF278021
:105C7F0053C2057F3F12DBD0C2057F0312DC10E455
:105C8F00900120F090018FF09001C7F090019BF0F0
:105C9F009001C6F090013CF07F0512DF277F0412C0
:105CAF00DF277F0312DF277F0212DF277F0112DF3B
:105CBF0027E4FF12DF279001C4E04402F07DFF7F4D
:105CCF000712DAEC9001C4E0FFC31330E046C205BF
:105CDF007F3F12DBD0C2057F0312DC10E49001205E
:105CEF00F090018FF09001C7F090019BF09001C6EA
:105CFF00F090013CF07F0512DF277F0412DF277F32
:105D0F000312DF277F0212DF277F0112DF27E4FF55
:105D1F0012DF27227F0112C92FEF640170749001E7
:105D2F008BE064017037C2057F4012DBD0C2057F64
:105D3F008012DBD0C2047F0112DBF0C2047F02129B
:105D4F00DBF0C2047F0412DBF0C2047F0812DBF029
:105D5F0090018B7402F07F0812DF278035D2057F08
:105D6F004012DBD0C2057F8012DBD0D2047F01123C
:105D7F00DBF0C2047F0212DBF0D2047F0412DBF0EF
:105D8F00C2047F0812DBF090018B7401F07F0812C0
:105D9F00D10D90018BE0B40103D38001C3403AC20F
:105DAF00057F4012DBD0C2057F8012DBD0C2047F9B
:105DBF000112DBF0C2047F0212DBF0C2047F041277
:105DCF00DBF0C2047F0812DBF090018B7402F07FCE
:105DDF000812DF277F0812DF277F0812C92FEF6411
:105DEF000160087F0812C92FBF0210D2057F011270
:105DFF00DC10C2057F0212DC108007C2057F011282
:105E0F00DC107F0912C92FEF640160087F0912C9E6
:105E1F002FBF0210D2057F0212DC10C2057F0112C4
:105E2F00DC108007C2057F0212DC107F0312C89CB2
:105E3F00EF6401600A7F0312C89CEF640270687FF1
:105E4F000412C89CEF640160087F0412C89CBF0253
:105E5F000EC2057F0212DBD0E49001C7F080619083
:105E6F0001C7E0601D7F0512C92FEF640160137F2A
:105E7F000512C92FEF640260097DFF7F0312DAEC70
:105E8F00803ED2057F0212DBD0C2057F0112DBD02C
:105E9F00E490019BF09001C774FFF07F0212DF279F
:105EAF007F0312D10D80197F0312C89CBF0411C24A
:105EBF00057F0212DBD0E49001C7F07F0312DF27CA
:105ECF007F0412C89CEF6401600A7F0412C89CEF24
:105EDF00640270687F0312C89CEF640160087F033F
:105EEF0012C89CBF020EC2057F0112DBD0E49001E5
:105EFF009BF0806190019BE0601D7F0512C92FEF21
:105F0F00640160137F0512C92FEF640260097DFFE2
:105F1F007F0212DAEC803ED2057F0112DBD0C20580
:105F2F007F0212DBD0E49001C7F090019B74FFF069
:105F3F007F0312DF277F0212D10D80197F0412C851
:105F4F009CBF0411C2057F0112DBD0E490019BF0CE
:105F5F007F0212DF277F0112C89CEF6401600A7F66
:105F6F000112C89CEF640270687F0212C89CEF6434
:105F7F000160087F0212C89CBF020EC2057F10127B
:105F8F00DBD0E4900120F08061900120E0601D7F64
:105F9F000612C92FEF640160137F0612C92FEF6439
:105FAF000260097DFF7F0512DAEC803ED2057F107B
:105FBF0012DBD0C2057F2012DBD0E490018FF0906E
:105FCF00012074FFF07F0412DF277F0512D10D80AF
:105FDF00197F0112C89CBF0411C2057F1012DBD0BC
:105FEF00E4900120F07F0512DF277F0212C89CEF9B
:105FFF006401600A7F0212C89CEF640270687F011F
:10600F0012C89CEF640160087F0112C89CBF020E8A
:10601F00C2057F2012DBD0E490018FF080619001E8
:10602F008FE0601D7F0612C92FEF640160137F069A
:10603F0012C92FEF640260097DFF7F0412DAEC8032
:10604F003ED2057F2012DBD0C2057F1012DBD0E4D9
:10605F00900120F090018F74FFF07F0512DF277FF2
:10606F000412D10D80197F0212C89CBF0411C20502
:10607F007F2012DBD0E490018FF07F0412DF277FA7
:10608F000512C89CEF6401600A7F0512C89CEF647B
:10609F000270747F0612C89CEF640160087F0612BD
:1060AF00C89CBF020EC2057F0812DBD0E49001C668
:1060BF00F0806D9001C6E060297F0412C92FEF6454
:1060CF0001601F7F0412C92FEF64026015C2057FA4
:1060DF000412DBD0E490013CF07DFF7F0112DAEC7B
:1060EF00803ED2057F0812DBD0C2057F0412DBD0C1
:1060FF00E490013CF09001C674FFF0E4FF12DF273B
:10610F007F0112D10D80197F0512C89CBF0411C2E7
:10611F00057F0812DBD0E49001C6F07F0112DF2764
:10612F007F0612C89CEF6401600A7F0612C89CEFBD
:10613F00640270737F0512C89CEF640160087F05CD
:10614F0012C89CBF020EC2057F0412DBD0E490017F
:10615F003CF0806B90013CE060287F0412C92FEF68
:10616F006401601E7F0412C92FEF64026014C20520
:10617F007F0812DBD0E49001C6F07DFFFF12DAEC4E
:10618F00803DD2057F0412DBD0C2057F0812DBD021
:10619F00E49001C6F090013C74FFF07F0112DF27FD
:1061AF00E4FF12D10D80187F0612C89CBF0410C2E5
:1061BF00057F0412DBD0E490013CF0FF12DF279043
:1061CF000188E064017027FF12C89CEF640160082A
:1061DF00E4FF12C89CBF02167F0212D3547F051230
:0F61EF00D10D7DFF7F0412DAECE4FF12D10D22F7
:10DD4E00300F08C20F12BD1C12DFB79001BCE0707D
:0ADD5E00087F031292F512E00F2275
:10AFB300300F3212DA90EF700302B12CC2A8C2AA8A
:10AFC300C20F12DEF47F0512DF477F0312D10D7D1E
:10AFD300FF7F0212DAEC7F0112D10D7F0312DEBF75
:10AFE3007F0512DEBF7F0312C89CBF010A12DB6319
:10AFF3007F0512DF4780607F0512C89CBF010A12DC
:10B00300DCAC7F0512DF47804E7F0412C89CEF64DF
:10B0130001704412DE5C7F0512DF4712E045EF60EA
:10B023001D7F0512D10D7DFF7F0412DAECE4FF12C0
:10B03300D10D7F0112DEBF7F0612DEBF80197F05AF
:10B0430012DF277F0412DF27E4FF12DF277F0112BD
:10B05300DF057F0612DF0512E045EF606C7F01120A
:10B06300C89CBF010A12D4037F031292F580107F9C
:10B073000612C89CBF010812D4577F031292F57FB2
:10B083000212C89CEF6401600302B12C12D29DBF6F
:10B09300011F7B017A01798E7D0412CD04400302E6
:10B0A300B12C7F0112D8FE7BFF7A9B79D612860CD6
:10B0B300229000D774FFF0A3749BF0A374E3F07B9A
:10B0C300017A01792912CA54227F0112C89CEF64C4
:10B0D30001600A7F0112C89CEF6402704C7F021268
:10B0E300C89CEF6401600A7F0212C89CEF6402707F
:10B0F300387F0612C89CEF640160087F0612C89C63
:10B10300BF0226E4FF12D3549000D374FFF0A3745C
:10B113009CF0A37431F07B017A01792912D0367F38
:0AB123000312DF057F0512DF05228D
:10003600E4900005F090002EF0A3F0200F030201DB
:10004600DB12DA90EF7003022674C20FD2A8E49096
:100056000175F0D2AA900176F090018BE0B401030D
:10006600D38001C34037C2057F4012DBD0C2057F73
:100076008012DBD0C2047F0112DBF0C2047F0212C1
:10008600DBF0C2047F0412DBF0C2047F0812DBF04F
:1000960090018B7402F07F0812DF278035D2057F2E
:1000A6004012DBD0C2057F8012DBD0D2047F011262
:1000B600DBF0C2047F0212DBF0D2047F0412DBF015
:1000C600C2047F0812DBF090018B7401F07F0812E6
:1000D600D10D900184E0FEA3E0FF12CDF8D390018C
:1000E60071E09FEE6480F8900170E06480984003B0
:1000F600020193900184E0FEA3E0FF12CDF8EF2405
:10010600FFFFEE34FFFEC3900171E09FEE6480F8BE
:10011600900170E06480984074900166E0FEA3E070
:10012600FFD3900174E09FEE6480F8900173E06461
:1001360080985059900121E0FEA3E0FFC374019F0F
:10014600FDE49EFC900184E0FAA3E0FBD39DEC6401
:1001560080F8EA6480985035C374FF9FFF74FF9E51
:10016600FEC3EB9FEE6480F8EA648098401F90011E
:10017600C4E04401F07F0612D10D7F0612D10D9026
:1001860001C4E04402F07DFF7F0712DAEC9001849F
:10019600E0FEA3E0FFD39401EE648094805012C386
:1001A600EF94FFEE6480947F40079001C4E044081A
:1001B600F0900184E0FEA3E0FFD3945BEE648094AC
:1001C600805012C3EF9459EE6480948040079001EA
:1001D600C4E04404F0900175E060030226749001C7
:1001E60076E0600302267412785650030226749055
:1001F600014DE024CDFF90014CE03400FE90015407
:10020600E0FCA3E0FD2FFFEC3EFEC3900145E09F1E
:10021600EE6480F8900144E064809850030203265F
:1002260090014DE0245AFF90014CE03400CF2DCFD1
:100236003CFEC390015BE09FEE6480F890015AE0BB
:100246006480985003020326E4FFFE12CDF8EF24E3
:100256006EFFE43EFE900144E0FCA3E0FDC39FEE8A
:100266006480F8EC6480985003020326900147E00E
:10027600246EFF900146E03400FEC3ED9FEE6480DD
:10028600F8EC6480985003020326900154E0FEA324
:10029600E0FF90014DE02FFF90014CE03EFEC39041
:1002A6000149E09FEE6480F8900148E06480984040
:1002B6006FE4FFFE12CDF890015AE0FCA3E0FDC307
:1002C6009FEE6480F8EC6480984055900146E0FE0D
:1002D600A3E0FFED9FEE6480F8EC6480984041E473
:1002E600FDFCFFFE1266F6C006C007E4FFFE12CD57
:1002F600F8D005D004C3ED9FEE6480F8EC648098D6
:10030600401EE4FDFCFFFE1266F6D3900147E09F17
:10031600EE6480F8900146E0648098500302073D41
:10032600C2057F3F12DBD0C2057F0312DC10E490CA
:100336000120F090018FF09001C7F090019BF090A2
:1003460001C6F090013CF07F0512DF277F0412DF23
:10035600277F0312DF277F0212DF277F0112DF27A5
:10036600E4FF12DF273010030205527B017A017980
:100376008E7D0412CD0440030226747F0412D8FE3B
:1003860090014DE024CDFF90014CE03400FE900139
:1003960055E02FFF900154E03EFEC3900145E09FDB
:1003A600EE6480F8900144E064809850329000EB4F
:1003B60074FFF0A3749CF0A374DBF0A374FFF0A3A6
:1003C600749CF0A374E1F0A374FFF0A3749CF0A3F3
:1003D60074F5F07B017A007906126C1302054890D9
:1003E600014DE0245AFF90014CE03400FE90015587
:1003F600E02FFF900154E03EFEC390015BE09FEECC
:100406006480F890015AE064809850329000EB7452
:10041600FFF0A3749CF0A374DBF0A374FFF0A37445
:100426009CF0A374E1F0A374FFF0A3749DF0A37491
:100436000FF07B017A007906126C13020548E4FF7F
:10044600FE12CDF8EF246EFFE43EFE900144E0FC80
:10045600A3E0FDC39FEE6480F8EC6480985003022D
:100466000519900147E0246EFF900146E03400FE36
:10047600C3ED9FEE6480F8EC648098500302051982
:10048600900154E0FEA3E0FF90014DE02FFF9001A4
:100496004CE03EFEC3900149E09FEE6480F8900177
:1004A60048E0648098406CE4FFFE12CDF890015A53
:1004B600E0FCA3E0FDC39FEE6480F8EC6480984006
:1004C60052900146E0FEA3E0FFED9FEE6480F8EC5B
:1004D600648098403EE4FDFCFFFE1266F6C006C04E
:1004E60007E4FFFE12CDF8D005D004C3ED9FEE64FD
:1004F60080F8EC648098401BE4FDFCFFFE1266F673
:10050600D3900147E09FEE6480F8900146E0648056
:1005160098402F9000EB74FFF0A3749CF0A374DB5B
:10052600F0A374FFF0A3749CF0A374E1F0A374FF2E
:10053600F0A3749DF0A37435F07B017A007906125E
:100546006C137B017A00790612860C22D20F900179
:1005560088E090013DF07B017A01798E7D0312CD12
:100566000440030226747F0412D8FE90014DE02455
:10057600CDFF90014CE03400FE900155E02FFF9036
:100586000154E03EFEC3900145E09FEE6480F89082
:100596000144E064809850329000EB74FFF0A3743D
:1005A6009CF0A374DBF0A374FFF0A3749CF0A37417
:1005B600E1F0A374FFF0A3749CF0A374F5F07B0143
:1005C6007A007906126C1302073390014DE0245A23
:1005D600FF90014CE03400FE900155E02FFF9001A2
:1005E60054E03EFEC390015BE09FEE6480F890010C
:1005F6005AE064809850329000EB74FFF0A3749C2C
:10060600F0A374DBF0A374FFF0A3749CF0A374E171
:10061600F0A374FFF0A3749DF0A3740FF07B017A2E
:10062600007906126C13020733E4FFFE12CDF8EFD1
:10063600246EFFE43EFE900144E0FCA3E0FDC39F70
:10064600EE6480F8EC64809850030207049001473A
:10065600E0246EFF900146E03400FEC3ED9FEE6499
:1006660080F8EC6480985003020704900154E0FE81
:10067600A3E0FF90014DE02FFF90014CE03EFEC34A
:10068600900149E09FEE6480F8900148E06480980C
:10069600406CE4FFFE12CDF890015AE0FCA3E0FDA9
:1006A600C39FEE6480F8EC6480984052900146E067
:1006B600FEA3E0FFED9FEE6480F8EC648098403E78
:1006C600E4FDFCFFFE1266F6C006C007E4FFFE125C
:1006D600CDF8D005D004C3ED9FEE6480F8EC6480BD
:1006E60098401BE4FDFCFFFE1266F6D3900147E03E
:1006F6009FEE6480F8900146E0648098402F900059
:10070600EB74FFF0A3749CF0A374DBF0A374FFF00A
:10071600A3749CF0A374E1F0A374FFF0A3749DF09E
:10072600A37435F07B017A007906126C137B017A8B
:1007360000790612860C229001C4E020E00302072D
:10074600EF900184E0FEA3E0FF12CDF8D390017193
:10075600E09FEE6480F8900170E0648098507B9092
:100766000184E0FEA3E0FF12CDF8EF24FCFFEE3497
:10077600FFFEC3900171E09FEE6480F8900170E087
:100786006480984055900166E0FEA3E0FFD3900197
:1007960074E09FEE6480F8900173E0648098503AAC
:1007A600900121E0FEA3E0FFC374019FFDE49EFCDF
:1007B600900184E0FAA3E0FBD39DEC6480F8EA6440
:1007C60080985016C374FF9FFF74FF9EFEC3EB9F75
:1007D600EE6480F8EA648098500F9001C4E054FEFD
:1007E600F07F0612D54F0209409001C4E030E003C5
:1007F6000209409001C6E0600302094090013CE016
:100806006003020940900184E0FEA3E0FF12CDF8E8
:10081600EF24FFFFEE34FFFED3900171E09FEE64FC
:1008260080F8900170E064809840030209409001CE
:1008360084E0FEA3E0FF12CDF8EF24FEFFEE34FFC6
:10084600FEC3900171E09FEE6480F8900170E06451
:1008560080985003020940900166E0FEA3E0FFD3B2
:10086600900174E09FEE6480F8900173E0648098D4
:100876004003020940900121E0FEA3E0FFC374019A
:100886009FFDE49EFC900184E0FAA3E0FBD39DEC7F
:100896006480F8EA6480984003020940C374FF9FAD
:1008A600FF74FF9EFEC3EB9FEE6480F8EA648098B7
:1008B6005003020940C2057F3F12DBD0C2057F0309
:1008C60012DC10E4900120F090018FF09001C7F047
:1008D60090019BF09001C6F090013CF07F0512DF7D
:1008E600277F0412DF277F0312DF277F0212DF270D
:1008F6007F0112DF27E4FF12DF279001C4E04401E5
:10090600F07F0612D10D7F0612D10D900184E0FE14
:10091600A3E0FFD39400EE64809480500FC3EE648E
:1009260080948040079001C4E04408F09001C4E040
:100936004402F07DFF7F0712DAEC9001C4E0FFC4A9
:1009460013540720E0030209E9900184E0FEA3E0C6
:10095600FFD3945DEE648094805079C3EF9457EE94
:1009660064809480406E900146E0FEA3E0FF24047C
:10097600FDE43EFC900170E0FAA3E0FBD39DEC643D
:1009860080F8EA648098504CEF24FEFFEE34FFFEB8
:10099600C3EB9FEE6480F8EA648098403790015676
:1009A600E0FEA3E0FF2403FDE43EFC900173E0FAC1
:1009B600A3E0FBD39DEC6480F8EA6480985015EFC1
:1009C60024FDFFEE34FFFEC3EB9FEE6480F8EA647D
:1009D6008098500F9001C4E054DFF07F0912D54F84
:1009E600020ADB9001C4E0FFC413540730E003029F
:1009F6000ADB900184E0FEA3E0FFD3945AEE648004
:100A060094804003020ADBC3EF945AEE648094801C
:100A16005003020ADB900147E02401FF900146E003
:100A26003400FE900170E0FCA3E0FDD39FEE6480ED
:100A3600F8EC6480984003020ADBC3ED9FEE648005
:100A4600F8EC6480985003020ADB900156E0FEA39E
:100A5600E0FF900173E0FCA3E0FDD39FEE6480F815
:100A6600EC648098506FC3ED9FEE6480F8EC648070
:100A7600984062C2057F3F12DBD0C2057F0312DCBD
:100A860010E4900120F090018FF09001C7F09001E2
:100A96009BF09001C6F090013CF07F0512DF277FA6
:100AA6000412DF277F0312DF277F0212DF277F0171
:100AB60012DF27E4FF12DF279001C4E04420F07F15
:100AC6000912D10D9001C4E04404F04402F07DFF08
:100AD6007F0712DAEC9001C4E0FF1313543F30E0B5
:100AE60024900184E0FCA3E0FDD3945CEC64809444
:100AF60080500BC3ED9458EC648094805007EF54FB
:100B0600FB9001C4F09001C4E0FF131313541F308F
:100B1600E024900184E0FCA3E0FDD39402EC648021
:100B26009480500BC3ED94FEEC6480947F5007EFE5
:100B360054F79001C4F09001C4E0FFC4540F30E0B4
:100B46002F7F0512C89CEF640160257F0512C89CA3
:100B5600EF6402601B7F0612C89CEF640160117F80
:100B66000612C89CEF640260079001C4E054EFF0DF
:100B76009001C5E0FF1313543F30E02F7F0412C8E5
:100B86009CEF640160257F0412C89CEF6402601B21
:100B96007F0312C89CEF640160117F0312C89CEFAB
:100BA600640260079001C5E054FBF0900152E0FE3C
:100BB600A3E0FF2404FDE43EFC900173E0FAA3E009
:100BC600FBD39DEC6480F8EA6480985015EF24FC12
:100BD600FFEE34FFFEC3EB9FEE6480F8EA64809874
:100BE60050079001C5E054F7F09001C4E0FFC4132C
:100BF60013540330E02F7F0812C92FEF64016025DC
:100C06007F0812C92FEF6402601B7F0912C92FEFFC
:100C1600640160117F0912C92FEF64026007900119
:100C2600C4E054BFF09001C4E0FFC4131313540191
:100C360030E024900121E0FCA3E0FDD39404EC64B1
:100C4600809480500BC3ED94FCEC6480947F500735
:100C5600EF547F9001C4F09001C5E0F930E0419077
:100C66000121E0FEA3E0FFC374049FFDE49EFC9017
:100C76000184E0FAA3E0FBD39DEC6480F8EA64808B
:100C8600985016C374FC9FFF74FF9EFEC3EB9FEE45
:100C96006480F8EA6480985007E954FE9001C5F034
:100CA600900120E06003020D4290018FE060030294
:100CB6000D429001C6E06003020D4290013CE070D7
:100CC6007B9001C7E0707590019BE0706F9001C446
:100CD600E030E01290019574FFF07F0612C1F2E455
:100CE600900195F0802C9001C4E0FFC413540730A6
:100CF600E01290019574FFF07F0712C1F2E49001B3
:100D060095F0800E90019574FFF012DC4FE490018F
:100D160095F09001C4E0FFC31330E0129001957482
:100D2600FFF07F0812C2ACE4900195F0800E9001AE
:100D36009574FFF012DC6EE4900195F07F0712C9FE
:100D46002FEF64016003020E699001C4E0FFC31334
:100D560020E003020E167F0112C89CEF64017003A7
:100D6600020E167F0112C89CEF64027003020E1673
:100D76007F0212C89CEF64017003020E167F0212F6
:100D8600C89CEF64027003020E167F0312C89CEF24
:100D96006401607C7F0312C89CEF640260727F046A
:100DA60012C89CEF640160687F0412C89CEF64025D
:100DB600605E7F0512C89CEF640160547F0512C80F
:100DC6009CEF6402604A7F0612C89CEF6401604093
:100DD6007F0612C89CEF64026036E4FF12C89CEFDF
:100DE6006401602CE4FF12C89CEF640260227F0756
:100DF60012C89CEF640160187F0712C89CEF64025A
:100E0600600E9001C4E054FDF07F0712DF27805387
:100E1600C2057F3F12DBD0C2057F0312DC10E490CF
:100E26000120F090018FF09001C7F090019BF090A7
:100E360001C6F090013CF07F0512DF277F0412DF28
:100E4600277F0312DF277F0212DF277F0112DF27AA
:100E5600E4FF12DF279001C4E04402F07DFF7F0724
:100E660012DAEC9001C4E0FFC31330E046C2057FFE
:100E76003F12DBD0C2057F0312DC10E4900120F0A4
:100E860090018FF09001C7F090019BF09001C6F0A1
:100E960090013CF07F0512DF277F0412DF277F03D6
:100EA60012DF277F0212DF277F0112DF27E4FF12FE
:100EB600DF2722D3900185E09400900184E06480CE
:100EC60094805003020FA67F0212C92FEF640160BF
:100ED6000D7F0212C92FEF64026003020FA6900174
:100EE600C5E0FFC31320E045C2057F3F12DBD0C239
:100EF600057F0312DC10E4900120F090018FF09042
:100F060001C7F090019BF09001C6F090013CF07F84
:100F16000512DF277F0412DF277F0312DF277F02F8
:100F260012DF277F0112DF27E4FF12DF277F01127E
:100F3600C89CEF6401600A7F0112C89CEF640270CE
:100F460046900184E0FEA3E0FF900121E0FCA3E0CF
:100F5600FD1266F6D3900171E09FEE6480F8900171
:100F660070E06480985020D2057F1012DBD0C20555
:100F76007F2012DBD0E490018FF090012074FFF007
:100F86007F0512D10D8011C2057F1012DBD0E490CF
:100F96000120F07F0512DF279001C5E04402F02210
:100FA6009001C5E0FFC31330E049EF54FDF0C205E0
:100FB6007F3F12DBD0C2057F0312DC10E4900120D4
:100FC600F090018FF09001C7F090019BF09001C660
:100FD600F090013CF07F0512DF277F0412DF277FA8
:100FE6000312DF277F0212DF277F0112DF27E4FFCC
:100FF60012DF27D3900185E09400900184E064809D
:101006009480407A7F0B12C92FEF6401600A7F0B30
:1010160012C92FEF640270669001C4E04410F0C25A
:10102600057F0812DBD0E49001C6F0C2057F0412EA
:10103600DBD0E490013CF090013EE0700ED2047FDC
:101046000112DBF0C2047F0212DBF0900196E07021
:101056000ED2057F4012DBD0C2057F8012DBD09016
:101066000192E0700ED2047F0412DBF0C2047F0806
:1010760012DBF090018B7401F07F0812D10D7F0115
:1010860012C92FEF6401600302112990018BE064FD
:1010960001704990013EE0700EC2047F0112DBF040
:1010A600C2047F0212DBF0900196E0700EC2057F4B
:1010B6004012DBD0C2057F8012DBD0900192E07037
:1010C6000EC2047F0412DBF0C2047F0812DBF0902C
:1010D600018B7402F07F0812DF27804790013EE003
:1010E600700ED2047F0112DBF0C2047F0212DBF025
:1010F600900196E0700ED2057F4012DBD0C2057FCC
:101106008012DBD0900192E0700ED2047F0412DBD5
:10111600F0C2047F0812DBF090018B7401F07F08A7
:1011260012D10D90019BE0F96024900167E0240A3A
:10113600FF900166E03400FED3900174E09FEE64F8
:1011460080F8900173E064809850030211ED9001DD
:10115600C7E0FF6021900169E024F6FD900168E098
:1011660034FFFCC3900174E09DEC6480F890017339
:10117600E064809850719001C5E0FE1313543F203F
:10118600E07BEF6030900152E0FEA3E0FF24F6FD25
:10119600EE34FFFC900173E0FAA3E0FBD39DEC6410
:1011A60080F8EA648098400DD3EB9FEE6480F8EAFD
:1011B6006480984032E96045900152E0FEA3E0FF6A
:1011C600240AFDE43EFC900173E0FAA3E0FBC39D14
:1011D600EC6480F8EA6480985023C3EB9FEE648049
:1011E600F8EA6480984016C2057F4012DBD0D2052B
:1011F6007F8012DBD090019674FFF08030E490017E
:1012060096F090018BE0B40103D38001C34010C275
:10121600057F4012DBD0C2057F8012DBD0800ED264
:10122600057F4012DBD0C2057F8012DBD09001C45F
:10123600E030E00302133D900166E0FEA3E0FFD339
:10124600900174E09FEE6480F8900173E0648098EA
:10125600400302133D900121E0FCA3E0FDC37401AD
:101266009DFBE49CFA900184E0FEA3E0FFD39BEA99
:101276006480F8EE648098400302133DC374FF9DBA
:10128600FD74FF9CFCC3EF9DEC6480F8EE648098CF
:10129600500302133D900120E0603C12CDF8EF248C
:1012A600FCFFEE34FFFED3900171E09FEE6480F800
:1012B600900170E0648098401E900184E0FEA3E0F7
:1012C600FF12CDF8D3900171E09FEE6480F8900193
:1012D60070E0648098404990018FE0605A900184E4
:1012E600E0FEA3E0FF12CDF8EF2404FFE43EFEC3C8
:1012F600900171E09FEE6480F8900170E064809840
:101306005035900184E0FEA3E0FF12CDF8C39001B2
:1013160071E09FEE6480F8900170E0648098401759
:10132600D2047F0412DBF0D2047F0812DBF09001B6
:101336009274FFF002170F900120E0603190018453
:10134600E0FEA3E0FF900121E0FCA3E0FD1266F6BB
:10135600EF24F6FFEE34FFFEC3900171E09FEE64CA
:1013660080F8900170E064809840030216C99001ED
:101376008FE06055D3900185E09400900184E0648D
:1013860080948040147F0B12C92FEF6401603A7F6E
:101396000B12C92FEF64026030900184E0FEA3E0D7
:1013A600FF900121E0FCA3E0FD1261FEEF240AFF9D
:1013B600E43EFED3900171E09FEE6480F8900170E8
:1013C600E064809850030216C99001C4E030E0033F
:1013D6000214C8900166E0FEA3E0FFD3900174E01A
:1013E6009FEE6480F8900173E064809840030214D5
:1013F600C8900121E0FCA3E0FDC374019DFBE49CC1
:10140600FA900184E0FEA3E0FFD39BEA6480F8EE45
:1014160064809840030214C8C374FF9DFD74FF9C4A
:10142600FCC3EF9DEC6480F8EE64809850030214D0
:10143600C8900120E0603F12CDF8EF24F6FFEE34AD
:10144600FFFED3900171E09FEE6480F8900170E09A
:101456006480984021900184E0FEA3E0FF12CDF85D
:10146600D3900171E09FEE6480F8900170E0648093
:101476009850030216C990018FE06046900184E0FF
:10148600FEA3E0FF12CDF8EF240AFFE43EFEC39070
:101496000171E09FEE6480F8900170E064809850DE
:1014A60021900184E0FEA3E0FF12CDF8C390017104
:1014B600E09FEE6480F8900170E06480984003023B
:1014C60016C99001C4E0FFC413540730E0030215A7
:1014D60097900184E0FEA3E0FFD3945AEE648094D3
:1014E600804003021597C3EF945AEE6480948050AF
:1014F60003021597900156E0FEA3E0FF900173E00A
:10150600FCA3E0FDD39FEE6480F8EC648098400372
:10151600021597C3ED9FEE6480F8EC6480984071E5
:10152600900120E06033900146E0FEA3E0FF24F640
:10153600FDEE34FFFC900170E0FAA3E0FBD39DECD6
:101546006480F8EA6480984010D3EB9FEE6480F8DC
:10155600EA64809850030216C990018FE0603290C9
:101566000146E0FEA3E0FF240AFDE43EFC90017084
:10157600E0FAA3E0FBC39DEC6480F8EA648098502F
:1015860010C3EB9FEE6480F8EA648098400302166D
:10159600C990013CE0F46003021634900120E0702B
:1015A6000990018FE07003021634900184E0FEA3D7
:1015B600E0FFD39400EE648094804072EF945AEE7C
:1015C600648094805068EF24FBFFEE34FFFE9001A8
:1015D60021E0FCA3E0FD1266F6900171E02414FD03
:1015E600900170E03400FCD3ED9FEE6480F8EC646B
:1015F600809840030216C9900185E024FBFF900104
:1016060084E034FFFE900121E0FCA3E0FD1261FEC0
:10161600900171E024ECFD900170E034FFFCC3ED15
:101626009FEE6480F8EC64809850030216C990011E
:10163600C6E0F460030216DF900120E07009900115
:101646008FE070030216DF900184E0FEA3E0FFC383
:10165600EE64809480400BD3EF945AEE64809480BD
:101666004077EF2405FFE43EFE900121E0FCA3E075
:10167600FD1266F6900171E02414FD900170E034CD
:1016860000FCD3ED9FEE6480F8EC648098503490B3
:101696000185E02405FF900184E03400FE900121DD
:1016A600E0FCA3E0FD1261FE900171E024ECFD90E8
:1016B6000170E034FFFCC3ED9FEE6480F8EC6480BB
:1016C600985016C2047F0412DBF0D2047F0812DBA6
:1016D600F090019274FFF08030E4900192F0900156
:1016E6008BE0B40103D38001C34010C2047F04120F
:1016F600DBF0C2047F0812DBF0800ED2047F0412F6
:10170600DBF0C2047F0812DBF09001C6E0F4600350
:101716000217EC900165E024F8FF900164E034FFC5
:10172600FE900184E0FCA3E0FDD39FEE6480F8EC1C
:1017360064809840030218C69001C4E0FF13131397
:10174600541F20E016C3EC64809480500EC3ED94C1
:10175600F8EC6480947F40030218C6EF1313543FDD
:1017660020E019C3ED945AEC64809480500EC3EDCA
:101776009452EC6480948040030218C6C3EC6480E3
:101786009480400BD3ED945AEC648094804057EDDE
:101796002405FFE43CFE900121E0FCA3E0FD126677
:1017A600F6D3900171E09FEE6480F8900170E064DA
:1017B600809840030218C6900185E02405FF900139
:1017C60084E03400FE900121E0FCA3E0FD1261FEFE
:1017D600C3900171E09FEE6480F8900170E0648030
:1017E6009850030218C690013CE0F460030218DC2E
:1017F60090015FE02408FF90015EE03400FE900156
:1018060084E0FCA3E0FDC39FEE6480F8EC6480985E
:1018160050030218C69001C4E0FF131313541F208F
:10182600E019D3ED9400EC64809480400ED3ED94DF
:1018360008EC6480948050030218C6EF1313543FDB
:1018460020E016D3ED945AEC64809480400BD3EDDF
:101856009462EC648094804067D3ED9400EC6480DD
:1018660094804072ED945AEC648094805068ED2424
:10187600FBFFEC34FFFE900121E0FCA3E0FD1266C5
:10188600F6D3900171E09FEE6480F8900170E064F9
:101896008098502C900185E024FBFF900184E03471
:1018A600FFFE900121E0FCA3E0FD1261FEC3900162
:1018B60071E09FEE6480F8900170E06480985016A5
:1018C600C2047F0112DBF0D2047F0212DBF090012A
:1018D6003E74FFF08030E490013EF090018BE0B45E
:1018E6000103D38001C34010C2047F0112DBF0C2A2
:1018F600047F0212DBF0800ED2047F0112DBF0C2FD
:10190600047F0212DBF09001C4E0FFC413135403FA
:1019160030E003021AF4900121E0FCA3E0FDD39429
:1019260000EC64809480502DC3EC64809480402544
:10193600EFC4131313540120E01BC2057F0112DC10
:1019460010C2057F0212DC109001C4E04480F0440E
:1019560040F0021B02900121E0FEA3E0FFC37401E8
:101966009FFDE49EFC900184E0FAA3E0FBD39DEC8E
:101976006480F8EA648098503CC374FF9FFF74FF4C
:101986009EFEC3EB9FEE6480F8EA64809840269042
:1019960001C5E020E01FC2057F0112DC10C2057FF1
:1019A6000212DC109001C5E04401F09001C4E0444D
:1019B60040F0021B027F0812C92FEF6401600D7F01
:1019C6000812C92FEF64026003021A4F90016EE0FD
:1019D600FEA3E0FF900121E0FCA3E0FDC39FEE64BF
:1019E60080F8EC6480985061900184E0FEA3E0FFEB
:1019F600ED2405FDE43CFC1266F6D3900171E09FF0
:101A0600EE6480F8900170E0648098503C90018408
:101A1600E0FEA3E0FF900122E02405FD900121E015
:101A26003400FC1261FEC3900171E09FEE6480F801
:101A3600900170E06480984010D2057F0112DC109E
:101A4600C2057F0212DC108007C2057F0112DC107E
:101A56007F0912C92FEF6401600D7F0912C92FEFAC
:101A660064026003021AEB90016AE0FEA3E0FF90B5
:101A76000121E0FCA3E0FDD39FEE6480F8EC6480D6
:101A8600984062900184E0FEA3E0FFED24FBFDECAC
:101A960034FFFC1266F6D3900171E09FEE6480F885
:101AA600900170E0648098503C900184E0FEA3E0D1
:101AB600FF900122E024FBFD900121E034FFFC129F
:101AC60061FEC3900171E09FEE6480F8900170E0C2
:101AD6006480984010D2057F0212DC10C2057F0197
:101AE60012DC108017C2057F0212DC10800EC205C0
:101AF6007F0112DC10C2057F0212DC109001C5E0E6
:101B0600FF1313543F30E003021C3B7F0312C89CB3
:101B1600EF6401600D7F0312C89CEF64026003024C
:101B26001C3B7F0412C89CEF640160087F0412C846
:101B36009CBF020FC2057F0212DBD0E49001C7F002
:101B4600021C4C900168E0FEA3E0FF900173E0FCEC
:101B5600A3E0FDC39FEE6480F8EC6480985030EDFE
:101B66009496EC648094804048900184E0FEA3E063
:101B7600FF900121E0FCA3E0FD1261FEC39001711C
:101B8600E09FEE6480F8900170E06480985022C275
:101B9600057F0212DBD0E49001C7F0C2057F011277
:101BA600DBD0E490019BF07DFF7F0312DAEC021C90
:101BB6004C9001C5E0FF131313541F20E05290010F
:101BC60052E0FEA3E0FF900173E0FCA3E0FDD39F8B
:101BD600EE6480F8EC6480985036C3ED9FEE648026
:101BE600F8EC6480984029C2057F0212DBD0E490AD
:101BF60001C7F0C2057F0112DBD0E490019BF07FA4
:101C06000312DF279001C5E04408F04404F0803653
:101C1600D2057F0212DBD0C2057F0112DBD0E49031
:101C2600019BF09001C774FFF07F0212DF277F034C
:101C360012D10D8011C2057F0212DBD0E49001C7DC
:101C4600F07F0312DF279001C5E0FF1313543F30E6
:101C5600E003021D547F0412C89CEF6401600D7FEF
:101C66000412C89CEF64026003021D547F0312C86D
:101C76009CEF640160087F0312C89CBF020FC20577
:101C86007F0112DBD0E490019BF0021D6590016696
:101C9600E0FEA3E0FFD3900174E09FEE6480F8902D
:101CA6000173E064809850227DFF7F0212DAECC255
:101CB600057F0212DBD0E49001C7F0C2057F011256
:101CC600DBD0E490019BF0021D659001C5E0FF1397
:101CD6001313541F20E052900152E0FEA3E0FF9040
:101CE6000173E0FCA3E0FDD39FEE6480F8EC648012
:101CF600985036C3ED9FEE6480F8EC6480984029D6
:101D0600C2057F0212DBD0E49001C7F0C2057F0155
:101D160012DBD0E490019BF07F0312DF279001C510
:101D2600E04408F04404F08036D2057F0112DBD08F
:101D3600C2057F0212DBD0E49001C7F090019B74CC
:101D4600FFF07F0312DF277F0212D10D8011C2053B
:101D56007F0112DBD0E490019BF07F0212DF277F28
:101D66000112C89CEF6401600D7F0112C89CEF64EC
:101D7600026003021DFC7F0212C89CEF640160082A
:101D86007F0212C89CBF020EC2057F1012DBD0E490
:101D9600900120F08071900184E0FEA3E0FF9001A5
:101DA60021E0FCA3E0FD1266F6C3900171E09FEE10
:101DB6006480F8900170E06480984015C2057F1039
:101DC60012DBD0E4900120F07DFF7F0512DAEC8073
:101DD60036D2057F1012DBD0C2057F2012DBD0E49D
:101DE60090018FF090012074FFF07F0412DF277FAF
:101DF6000512D10D8011C2057F1012DBD0E49001CF
:101E060020F07F0512DF277F0212C89CEF64016075
:101E16000D7F0212C89CEF64026003021EB07F01B0
:101E260012C89CEF640160087F0112C89CBF020EB5
:101E3600C2057F2012DBD0E490018FF0807D9001F7
:101E460084E0FEA3E0FF900121E0FCA3E0FD126127
:101E5600FED3900171E09FEE6480F8900170E0641B
:101E660080985021C2057F2012DBD0E490018FF0CC
:101E7600C2057F1012DBD0E4900120F07DFF7F04C5
:101E860012DAEC8036D2057F2012DBD0C2057F1035
:101E960012DBD0E4900120F090018F74FFF07F05F3
:101EA60012DF277F0412D10D8011C2057F2012DBBD
:101EB600D0E490018FF07F0412DF279001C4E0FF89
:101EC600C4540F30E00302205E7F0512C89CEF6405
:101ED60001600D7F0512C89CEF6402600302205E5C
:101EE6007F0612C89CEF640160087F0612C89CBF7B
:101EF600020FC2057F0812DBD0E49001C6F0022073
:101F06006F900164E0FEA3E0FF900184E0FCA3E093
:101F1600FDC39FEE6480F8EC6480985051ED240573
:101F2600FFE43CFE900121E0FCA3E0FD1266F6D33F
:101F3600900171E09FEE6480F8900170E0648098F3
:101F4600502C900185E02405FF900184E03400FECA
:101F5600900121E0FCA3E0FD1261FEC3900171E057
:101F66009FEE6480F8900170E06480985022C2056C
:101F76007F0812DBD0E49001C6F0C2057F0412DBB5
:101F8600D0E490013CF07DFF7F0112DAEC02206F75
:101F96009001C4E0FF1313543F20E047900184E012
:101FA600FEA3E0FFD3945AEE648094805035C3EFCD
:101FB600945AEE64809480402AC2057F0812DBD0D2
:101FC600E49001C6F0C2057F0412DBD0E490013C28
:101FD600F07F0112DF279001C4E04404F04410F0C2
:101FE60002206F9001C4E0FF131313541F20E04337
:101FF600900184E0FEA3E0FFD39400EE6480948019
:102006005031C3EE648094804029C2057F0812DBFC
:10201600D0E49001C6F0C2057F0412DBD0E4900143
:102026003CF07F0112DF279001C4E04408F0441021
:10203600F08036D2057F0812DBD0C2057F0412DBA2
:10204600D0E490013CF09001C674FFF0E4FF12DF8B
:10205600277F0112D10D8011C2057F0812DBD0E463
:102066009001C6F07F0112DF279001C4E0FFC4543F
:102076000F30E00302220B7F0612C89CEF6401605A
:102086000D7F0612C89CEF6402600302220B7F05D7
:1020960012C89CEF640160087F0512C89CBF020F3E
:1020A600C2057F0412DBD0E490013CF002221B90B3
:1020B600015EE0FEA3E0FF900184E0FCA3E0FDD317
:1020C6009FEE6480F8EC6480984052ED24FBFFECB0
:1020D60034FFFE900121E0FCA3E0FD1266F6D390EA
:1020E6000171E09FEE6480F8900170E06480985082
:1020F6002C900185E024FBFF900184E034FFFE90E4
:102106000121E0FCA3E0FD1261FEC3900171E09F96
:10211600EE6480F8900170E06480985021C2057FDB
:102126000412DBD0E490013CF0C2057F0812DBD03C
:10213600E49001C6F07DFFFF12DAEC02221B90014B
:10214600C4E0FF1313543F20E046900184E0FEA351
:10215600E0FFD3945AEE648094805034C3EF945ACF
:10216600EE648094804029C2057F0812DBD0E4909B
:1021760001C6F0C2057F0412DBD0E490013CF0FFFB
:1021860012DF279001C4E04404F04410F002221B41
:102196009001C4E0FF131313541F20E04390018401
:1021A600E0FEA3E0FFD39400EE648094805031C338
:1021B600EE648094804029E4FF12DF27C2057F0881
:1021C60012DBD0E49001C6F0C2057F0412DBD0E436
:1021D60090013CF09001C4E04408F04410F08035D2
:1021E600D2057F0412DBD0C2057F0812DBD0E49053
:1021F60001C6F090013C74FFF07F0112DF27E4FF77
:1022060012D10D8010C2057F0412DBD0E490013C90
:10221600F0FF12DF27E4FF12C89CEF6401600DE4B3
:10222600FF12C89CEF640260030223827F0712C874
:102236009CEF640170030223827F0712C89CEF643F
:102246000270030223827F0712C92FEF6401700315
:102256000223827F0712C92FEF64027003022382D2
:102266007F0112C89CEF640170030223827F011272
:10227600C89CEF640270030223827F0212C89CEF9F
:10228600640170030223827F0212C89CEF6402700D
:10229600030223827F0512C89CEF640170030223A8
:1022A600827F0512C89CEF640270030223827F06B8
:1022B60012C89CEF640170030223827F0612C89C39
:1022C600EF640270030223827F0412C89CEF64014C
:1022D60070030223827F0412C89CEF64027003021B
:1022E60023827F0312C89CEF640170030223827F5E
:1022F6000312C89CEF640270030223827F0112C995
:102306002FEF640160767F0112C92FEF6402606CC3
:10231600E49001C2F0A3F0900166E0FFA3E0900113
:1023260097CFF0A3EFF0E4FFFE12CDF8900193EE05
:10233600F0A3EFF0E4900135F0A3F09001C4E0546F
:10234600FEF07F0612D54F9001C4E054DFF07F09FE
:1023560012D54F9001C4E04401F07F0612D10D7FE3
:102366000612D3549000D374FFF0A3749CF0A374A8
:1023760031F07B017A01792912D036227F0712C803
:102386009CEF6401600D7F0712C89CEF6402600336
:102396000224EEE4FF12C89CEF640170030224EEEF
:1023A600E4FF12C89CEF640270030224EE7F07125A
:1023B600C92FEF640170030224EE7F0712C92FEFC5
:1023C600640270030224EE7F0112C89CEF64017060
:1023D600030224EE7F0112C89CEF640270030224FC
:1023E600EE7F0212C89CEF640170030224EE7F02A6
:1023F60012C89CEF640270030224EE7F0512C89C8B
:10240600EF640170030224EE7F0512C89CEF64029C
:1024160070030224EE7F0612C89CEF64017003026B
:1024260024EE7F0612C89CEF640270030224EE7F3E
:102436000412C89CEF640170030224EE7F0412C8E4
:102446009CEF640270030224EE7F0312C89CEF64C3
:102456000170030224EE7F0312C89CEF640270032E
:102466000224EE7F0112C92FEF6401607B7F011207
:10247600C92FEF640260719001C2E4F0A3745AF0B0
:10248600900156E0FFA3E0900197CFF0A3EFF09004
:102496000146E0FFA3E0900193CFF0A3EFF0900197
:1024A60035E4F0A37407F09001C4E054FEF07F0613
:1024B60012D54F9001C4E054DFF07F0912D54F903A
:1024C60001C4E04420F07F0912D10D7F0612D354D7
:1024D6009000D374FFF0A3749CF0A37431F07B01D9
:1024E6007A01792912D036222010030226747F0140
:1024F60012C89CEF6401600D7F0112C89CEF640254
:1025060060030225BC7F0312C89CEF6401600D7F47
:102516000312C89CEF640260030225BC7F0712C841
:102526009CEF640170030225BC7F0712C89CEF6410
:102536000270030225BC7F0412C89CEF640160761A
:102546007F0412C89CEF6402606CE4FF12C89CEF23
:1025560064016062E4FF12C89CEF640260587F0267
:1025660012C89CEF6401604E7F0212C89CEF6402A1
:1025760060447F0512C89CEF6401603A7F0512C86B
:102586009CEF640260307F0612C89CEF64016026EF
:102596007F0612C89CEF6402601C7F0712D354901A
:1025A60000D774FFF0A3749BF0A374D2F07B017A7A
:1025B60001792912CA547F0312C89CEF6401600A8C
:1025C6007F0312C89CEF640270457F0412C89CEF1B
:1025D6006401600A7F0412C89CEF640270317F05B3
:1025E60012C89CEF640160087F0512C89CBF021FD9
:1025F6007F0312D35412BF979000D374FFF0A374D5
:102606009DF0A3745AF07B017A01792912D0367FA6
:102616000112C89CEF6401600A7F0112C89CEF6436
:1026260002704B7F0212C89CEF6401600A7F02129F
:10263600C89CEF640270377F0612C89CEF64016085
:10264600087F0612C89CBF02257F0212D35412BF10
:10265600979000D374FFF0A3749DF0A3745EF07B93
:0E266600017A01792912D03690018A74FFF0B2
:012674002243
:1033BF00200F030234FE900136E0FF12C89CEF6429
:1033CF00016010900136E0FF12C89CEF64026003A9
:1033DF000234B3D2A8E4900175F0D2AA900176F02E
:1033EF00C20F900125F012BF9790018BE06401701E
:1033FF0037D2057F4012DBD0C2057F8012DBD0D2DF
:10340F00047F0112DBF0C2047F0212DBF0D2047FD3
:10341F000412DBF0C2047F0812DBF090018B740101
:10342F00F07F0812D10D8035C2057F4012DBD0C26C
:10343F00057F8012DBD0C2047F0112DBF0C2047F54
:10344F000212DBF0C2047F0412DBF0C2047F081209
:10345F00DBF090018B7402F07F0812DF27C2057F2B
:10346F003F12DBD0C2057F0312DC10E4900120F085
:10347F0090018FF09001C7F090019BF09001C6F082
:10348F0090013CF07F0512DF277F0412DF277F03B7
:10349F0012DF277F0212DF277F0112DF27E4FF12DF
:1034AF00DF27804BC2057F3F12DBD0C2057F03129F
:1034BF00DC10E4900120F090018FF09001C7F090A4
:1034CF00019BF09001C6F090013CF07F0512DF27C1
:1034DF007F0412DF277F0312DF277F0212DF277F90
:1034EF000112DF27E4FF12DF27E4FF12D3542290EB
:1034FF000136E0FF12C89CEF64016058900136E07E
:10350F00FF12C89CEF6402604BC2057F3F12DBD0F5
:10351F00C2057F0312DC10E4900120F090018FF0C0
:10352F009001C7F090019BF09001C6F090013CF024
:10353F007F0512DF277F0412DF277F0312DF277F2C
:10354F000212DF277F0112DF27E4FF12DF27E4FFDC
:10355F0012D354227F0712C92FEF6401600A900122
:10356F00C4E0FFC31330E059E4FF12D354C2057F08
:10357F003F12DBD0C2057F0312DC10E4900120F074
:10358F0090018FF09001C7F090019BF09001C6F071
:10359F0090013CF07F0512DF277F0412DF277F03A6
:1035AF0012DF277F0212DF277F0112DF27E4FF12CE
:1035BF00DF279001C4E04402F07DFF7F0712DAECB1
:1035CF00221278565003023F0DD3900185E09400EC
:1035DF00900184E06480948040147F0B12C92FEF18
:1035EF006401602F7F0B12C92FEF64026025D39007
:1035FF000185E09400900184E064809480406D7FA9
:10360F000212C92FEF6401600A7F0212C92FEF6403
:10361F00027059C2057F3F12DBD0C2057F0312DC57
:10362F0010E4900120F090018FF09001C7F090010D
:10363F009BF09001C6F090013CF07F0512DF277FD1
:10364F000412DF277F0312DF277F0212DF277F019C
:10365F0012DF27E4FF12DF279001C4E04402F07D60
:10366F00FF7F0712DAECE4FF12D35422900197E0A8
:10367F00FEA3E0FF900173E0B50620A3E0B5071BA2
:10368F00C2057F0212DBD0E49001C7F0C2057F01B3
:10369F0012DBD0E490019BF00237AC900197E0FE73
:1036AF00A3E0FF24F6FDEE34FFFC900173E0FAA3D4
:1036BF00E0FBC39DEC6480F8EA648098402AEF2415
:1036CF000AFFE43EFED3EB9FEE6480F8EA64809835
:1036DF005016C2057F4012DBD0D2057F8012DBD09F
:1036EF0090019674FFF08005E4900196F090019799
:1036FF00E0FEA3E0FF900173E0FCA3E0FDD39FEE9B
:10370F006480F8EC6480984030900166E0FEA3E09E
:10371F00FFD3ED9FEE6480F8EC648098401BD205D8
:10372F007F0112DBD0C2057F0212DBD0E49001C70C
:10373F00F090019B74FFF08064900197E0FEA3E08E
:10374F00FF900173E0FCA3E0FDC39FEE6480F8ECF3
:10375F006480985030900168E0FEA3E0FFC3ED9FB6
:10376F00EE6480F8EC648098501BD2057F0212DB68
:10377F00D0C2057F0112DBD0E490019BF09001C70E
:10378F0074FFF08018C2057F0212DBD0E49001C7EE
:10379F00F0C2057F0112DBD0E490019BF090012174
:1037AF00E0FEA3E0FFC3EE64809480400302383D47
:1037BF0090016EE0FCA3E0FDC3EF9DEC6480F8EE9A
:1037CF006480985069900184E0FEA3E0FF9001228D
:1037DF00E02405FD900121E03400FC1266F6D39041
:1037EF000171E09FEE6480F8900170E06480985062
:1037FF003D900184E0FEA3E0FF900122E02405FD4F
:10380F00900121E03400FC1261FEC3900171E09F32
:10381F00EE6480F8900170E06480984011D2057FCB
:10382F000112DC10C2057F0212DC100238DD90019C
:10383F0021E0FEA3E0FFD39400EE64809480500358
:10384F000238CF90016AE0FCA3E0FDD3EF9DEC645A
:10385F0080F8EE6480984068900184E0FEA3E0FF5A
:10386F00900122E024FBFD900121E034FFFC126661
:10387F00F6D3900171E09FEE6480F8900170E064E0
:10388F008098503C900184E0FEA3E0FF900122E07D
:10389F0024FBFD900121E034FFFC1261FEC3900177
:1038AF0071E09FEE6480F8900170E06480984010A2
:1038BF00D2057F0212DC10C2057F0112DC10800ED0
:1038CF00C2057F0112DC10C2057F0212DC109001CD
:1038DF0025E07003023AA8C2057F0812DBD0E490FE
:1038EF0001C6F0C2057F0412DBD0E490013CF090DA
:1038FF000193E0FEA3E0FF24FCFDEE34FFFC9001FA
:10390F0070E0FAA3E0FBC39DEC6480F8EA64809852
:10391F00402AEF2404FFE43EFED3EB9FEE6480F8D1
:10392F00EA6480985016D2047F0412DBF0D2047F31
:10393F000812DBF090019274FFF08077900193E012
:10394F00FEA3E0FF24F6FDEE34FFFC900170E0FAD9
:10395F00A3E0FBC39DEC6480F8EA648098402AEFF3
:10396F00240AFFE43EFED3EB9FEE6480F8EA648006
:10397F00985016C2047F0412DBF0D2047F0812DBCA
:10398F00F090019274FFF0802AE4900192F0900180
:10399F008BE0B40110D2047F0412DBF0C2047F0865
:1039AF0012DBF0800EC2047F0412DBF0C2047F082A
:1039BF0012DBF0900194E024FFFF900193E034FFBD
:1039CF00FEC3900171E09FEE6480F8900170E06497
:1039DF0080985048900184E0FEA3E0FF900121E021
:1039EF00FCA3E0FD1266F6C3900171E09FEE6480C8
:1039FF00F8900170E06480984003D38001C3401CAD
:103A0F00D2057F1012DBD0C2057F2012DBD0E490ED
:103A1F00018FF090012074FFF0023DA3900193E01D
:103A2F00FEA3E0FFD3900171E09FEE6480F8900158
:103A3F0070E06480984047900184E0FEA3E0FF901F
:103A4F000121E0FCA3E0FD1261FED3900171E09F24
:103A5F00EE6480F8900170E064809850028001C39A
:103A6F00401CD2057F2012DBD0C2057F1012DBD0A5
:103A7F00E4900120F090018F74FFF0023DA3C20586
:103A8F007F1012DBD0E4900120F0C2057F2012DB03
:103A9F00D0E490018FF0023DA39001C2E0FEA3E0BD
:103AAF00FF24F6FDEE34FFFC900184E0FAA3E0FB67
:103ABF00C39DEC6480F8EA648098402AEF240AFFE3
:103ACF00E43EFED3EB9FEE6480F8EA6480985016D4
:103ADF00C2047F0112DBF0D2047F0212DBF09001EF
:103AEF003E74FFF08005E490013EF0E4FDFCFFFE24
:103AFF001266F6C3900171E09FEE6480F89001703A
:103B0F00E06480984022E4FDFCFFFE1266F6EF248D
:103B1F000AFFE43EFED3900171E09FEE6480F890BF
:103B2F000170E0648098403EE4FDFCFFFE1261FEF0
:103B3F00D3900171E09FEE6480F8900170E0648093
:103B4F00985039E4FDFCFFFE1261FEEF24F6FFEE04
:103B5F0034FFFEC3900171E09FEE6480F890017016
:103B6F00E06480984016C2047F0412DBF0D2047F19
:103B7F000812DBF090019274FFF08005E49001923F
:103B8F00F09001C2E0FEA3E0FF900184E06E7003AD
:103B9F00A3E06F7039C2057F0812DBD0E49001C635
:103BAF00F0C2057F0412DBD0E490013CF0C2057F28
:103BBF002012DBD0E490018FF0C2057F1012DBD012
:103BCF00E4900120F090012574FFF0023DA3E4FD85
:103BDF00FCFFFE1266F6C3900171E09FEE6480F861
:103BEF00900170E0648098405FC2057F0812DBD0BF
:103BFF00E49001C6F0C2057F0412DBD0E490013CD3
:103C0F00F0900184E0FEA3E0FF900121E0FCA3E02F
:103C1F00FD1261FED3900171E09FEE6480F8900178
:103C2F0070E064809850028001C34007D2057F2066
:103C3F0012DBD0C2057F1012DBD0E4900120F09090
:103C4F00018F74FFF0023DA3E4FDFCFFFE1261FE45
:103C5F00D3900171E09FEE6480F8900170E0648072
:103C6F00985060C2057F0812DBD0E49001C6F0C205
:103C7F00057F0412DBD0E490013CF0900184E0FE5C
:103C8F00A3E0FF900121E0FCA3E0FD1266F6C390D4
:103C9F000171E09FEE6480F8900170E064809840BD
:103CAF0003D38001C34007D2057F1012DBD0C205BA
:103CBF007F2012DBD0E490018FF090012074FFF091
:103CCF00023DA39001C2E0FEA3E0FF900184E0FC5F
:103CDF00A3E0FDD39FEE6480F8EC648098404D9094
:103CEF00015EE0FEA3E0FFD3ED9FEE6480F8EC648D
:103CFF00809850028001C34033C2057F2012DBD071
:103D0F00E490018FF0C2057F1012DBD0E490012008
:103D1F00F0D2057F0412DBD0C2057F0812DBD0E49E
:103D2F009001C6F090013C74FFF080689001C2E0F2
:103D3F00FEA3E0FF900184E0FCA3E0FDC39FEE64CF
:103D4F0080F8EC648098504C900164E0FEA3E0FF93
:103D5F00C3ED9FEE6480F8EC6480984003D380013C
:103D6F00C34031C2057F2012DBD0E490018FF0C237
:103D7F00057F1012DBD0E4900120F0D2057F0812EE
:103D8F00DBD0C2057F0412DBD0E490013CF0900140
:103D9F00C674FFF07F0112C92FEF64016003023E6A
:103DAF004890018BE06401704990013EE0700EC2B3
:103DBF00047F0112DBF0C2047F0212DBF090019648
:103DCF00E0700EC2057F4012DBD0C2057F8012DB90
:103DDF00D0900192E0700EC2047F0412DBF0C20497
:103DEF007F0812DBF090018B7402F07F0812DF273F
:103DFF00804790013EE0700ED2047F0112DBF0C2CB
:103E0F00047F0212DBF0900196E0700ED2057F4026
:103E1F0012DBD0C2057F8012DBD0900192E0700ED2
:103E2F00D2047F0412DBF0C2047F0812DBF0900192
:103E3F008B7401F07F0812D10D900197E0FEA3E083
:103E4F00FF900173E06E7003A3E06F6003023F0DFC
:103E5F009001C2E0FEA3E0FF900184E06E7003A327
:103E6F00E06F6003023F0D900193E0FEA3E0FF902F
:103E7F000170E0FCA3E0FDD39FEE6480F8EC64805A
:103E8F0098507BEF24FFFFEE34FFFEC3ED9FEE64EF
:103E9F0080F8EC6480984066900121E07002A3E006
:103EAF00705CC2057F3F12DBD0C2057F0312DC10AE
:103EBF00E4900120F090018FF09001C7F090019BEA
:103ECF00F09001C6F090013CF07F0512DF277F04D0
:103EDF0012DF277F0312DF277F0212DF277F0112F6
:103EEF00DF27E4FF12DF279001C4E04402F07DFFDB
:0F3EFF007F0712DAECE4900125F0FF12D3542272
:104978009001C4E04402F07DFF7F0712DAEC7F0863
:1049880012D10D90019BE06021900167E0240AFF9D
:10499800900166E03400FED3900174E09FEE6480DD
:1049A800F8900173E064809840279001C7E0603771
:1049B800900169E024F6FF900168E034FFFEC3909F
:1049C8000174E09FEE6480F8900173E06480984081
:1049D80016C2057F4012DBD0D2057F8012DBD09053
:1049E800019674FFF08013E4900196F0D2057F40A1
:1049F80012DBD0C2057F8012DBD0900120E060314D
:104A0800900184E0FEA3E0FF900121E0FCA3E0FD1B
:104A18001266F6EF24F6FFEE34FFFEC3900171E054
:104A28009FEE6480F8900170E06480984003024B28
:104A3800C690018FE06055D3900185E09400900105
:104A480084E06480948040147F0B12C92FEF6401C6
:104A5800603A7F0B12C92FEF64026030900184E046
:104A6800FEA3E0FF900121E0FCA3E0FD1261FEEF50
:104A7800240AFFE43EFED3900171E09FEE6480F8C3
:104A8800900170E06480985003024BC690013CE0AE
:104A9800F46003024B31900120E0700990018FE02F
:104AA8007003024B31900184E0FEA3E0FFD3940031
:104AB800EE648094804072EF945AEE648094805043
:104AC80068EF24FBFFEE34FFFE900121E0FCA3E039
:104AD800FD1266F6900171E02414FD900170E03437
:104AE80000FCD3ED9FEE6480F8EC648098400302EC
:104AF8004BC6900185E024FBFF900184E034FFFE63
:104B0800900121E0FCA3E0FD1261FE900171E02418
:104B1800ECFD900170E034FFFCC3ED9FEE6480F87B
:104B2800EC6480985003024BC69001C6E0F4600321
:104B3800024BDC900120E0700990018FE0700302C5
:104B48004BDC900184E0FEA3E0FFC3EE6480948018
:104B5800400BD3EF945AEE648094804077EF24059D
:104B6800FFE43EFE900121E0FCA3E0FD1266F69012
:104B78000171E02414FD900170E03400FCD3ED9F36
:104B8800EE6480F8EC6480985034900185E0240548
:104B9800FF900184E03400FE900121E0FCA3E0FDD9
:104BA8001261FE900171E024ECFD900170E034FF89
:104BB800FCC3ED9FEE6480F8EC6480985016C20444
:104BC8007F0412DBF0D2047F0812DBF090019274AC
:104BD800FFF08013E4900192F0D2047F0412DBF01E
:104BE800C2047F0812DBF0D2047F0112DBF0C2049A
:104BF8007F0212DBF07F0812D10D90013BE06003C9
:104C0800024E1E9001BDE06003024E1E900183E03B
:104C180030E54A900184E0FEA3E0FF900121E0FC2A
:104C2800A3E0FD1266F6D3900171E09FEE6480F870
:104C3800900170E06480985024D2057F1012DBD078
:104C4800C2057F2012DBD0E490018FF09001207420
:104C5800FFF012DFC490013B74FFF080699001837C
:104C6800E030E44A900184E0FEA3E0FF900121E0F7
:104C7800FCA3E0FD1261FEC3900171E09FEE648029
:104C8800F8900170E06480984024D2057F2012DB00
:104C9800D0C2057F1012DBD0E4900120F090018F84
:104CA80074FFF012DFC490013B74FFF08018C20556
:104CB8007F1012DBD0E4900120F0C2057F2012DBC8
:104CC800D0E490018FF0900183E020E303024D6B64
:104CD80090015EE0FEA3E0FF900184E0FCA3E0FD0C
:104CE800D39FEE6480F8EC6480984077ED24FBFF56
:104CF800EC34FFFE900121E0FCA3E0FD1266F6D340
:104D0800900171E09FEE6480F8900170E0648098F3
:104D18005051900185E024FBFF900184E034FFFEB0
:104D2800900121E0FCA3E0FD1261FEC3900171E057
:104D38009FEE6480F8900170E06480984025D20569
:104D48007F0412DBD0C2057F0812DBD0E49001C6D5
:104D5800F090013C74FFF012DFC490013B74FFF047
:104D6800024E1E900183E020E203024E0690016489
:104D7800E0FEA3E0FF900184E0FCA3E0FDC39FEE0A
:104D88006480F8EC6480985075ED2405FFE43CFEDF
:104D9800900121E0FCA3E0FD1266F6D3900171E0DA
:104DA8009FEE6480F8900170E06480985050900104
:104DB80085E02405FF900184E03400FE900121E0A5
:104DC800FCA3E0FD1261FEC3900171E09FEE6480D8
:104DD800F8900170E06480984024D2057F0812DBC7
:104DE800D0C2057F0412DBD0E490013CF09001C6EC
:104DF80074FFF012DFC490013B74FFF08018C20505
:104E08007F0812DBD0E49001C6F0C2057F0412DBF4
:104E1800D0E490013CF07F0712C92FEF6401600DC8
:104E28007F0712C92FEF640260030251827F0812C4
:104E3800D10D7F0712D10D7F0112C89CEF6401606C
:104E48000A7F0112C89CEF6402704C900184E0FE56
:104E5800A3E0FF900121E0FCA3E0FD1266F6C390F9
:104E68000171E09FEE6480F8900170E064809840E2
:104E780003D38001C34020D2057F1012DBD0C205C6
:104E88007F2012DBD0E490018FF090012074FFF0B6
:104E98007F0512D10D8011C2057F1012DBD0E4907E
:104EA8000120F07F0512DF277F0212C89CEF640102
:104EB800600A7F0212C89CEF6402704B900184E084
:104EC800FEA3E0FF900121E0FCA3E0FD1261FED308
:104ED800900171E09FEE6480F8900170E064809822
:104EE80050028001C34020D2057F2012DBD0C205CA
:104EF8007F1012DBD0E4900120F090018F74FFF056
:104F08007F0412D10D8011C2057F2012DBD0E490FE
:104F1800018FF07F0412DF277F0512C89CEF640120
:104F2800600D7F0512C89CEF64026003024FC490B5
:104F38000164E0FEA3E0FF900184E0FCA3E0FDC370
:104F48009FEE6480F8EC6480985071ED2405FFE4CE
:104F58003CFE900121E0FCA3E0FD1266F6D390012F
:104F680071E09FEE6480F8900170E0648098504C86
:104F7800900185E02405FF900184E03400FE900153
:104F880021E0FCA3E0FD1261FEC3900171E09FEEF9
:104F98006480F8900170E06480984020D2057F0812
:104FA80012DBD0C2057F0412DBD0E490013CF09004
:104FB80001C674FFF07F0112D10D8011C2057F0870
:104FC80012DBD0E49001C6F07F0112DF277F0612C2
:104FD800C89CEF6401600D7F0612C89CEF640260F4
:104FE8000302507A90015EE0FEA3E0FF900184E0A6
:104FF800FCA3E0FDD39FEE6480F8EC6480984072D7
:10500800ED24FBFFEC34FFFE900121E0FCA3E0FD62
:105018001266F6D3900171E09FEE6480F8900170FB
:10502800E0648098504C900185E024FBFF90018457
:10503800E034FFFE900121E0FCA3E0FD1261FEC315
:10504800900171E09FEE6480F8900170E0648098B0
:105058004020D2057F0412DBD0C2057F0812DBD0C6
:10506800E49001C6F090013C74FFF0E4FF12D10D0A
:105078008010C2057F0412DBD0E490013CF0FF12DF
:10508800DF277F0312C89CEF6401600A7F0312C800
:105098009CEF6402706C900168E0FEA3E0FF900151
:1050A80073E0FCA3E0FDC39FEE6480F8EC64809895
:1050B8005050ED9496EC648094804026900184E0F2
:1050C800FEA3E0FF900121E0FCA3E0FD1261FEC316
:1050D800900171E09FEE6480F8900170E064809820
:1050E8004020D2057F0212DBD0C2057F0112DBD03F
:1050F800E490019BF09001C774FFF07F0312D10D7B
:105108008011C2057F0212DBD0E49001C7F07F0353
:1051180012DF277F0412C89CEF6401600A7F041223
:10512800C89CEF64027040900166E0FEA3E0FFD3E4
:10513800900174E09FEE6480F8900173E0648098B9
:1051480050028001C34020D2057F0112DBD0C20586
:105158007F0212DBD0E49001C7F090019B74FFF04E
:105168007F0212D10D805EC2057F0112DBD0E49070
:10517800019BF07F0212DF27804B90013BE07045D6
:10518800C2057F3F12DBD0C2057F0312DC10E4901A
:105198000120F090018FF09001C7F090019BF090F2
:1051A80001C6F090013CF07F0512DF277F0412DF73
:1051B800277F0312DF277F0212DF277F0112DF27F5
:1051C800E4FF12DF2790013BE060219001BDE0C3BE
:1051D80094645018C2057F0812DBD0E49001C6F031
:1051E800C2057F0412DBD0E490013CF090013BE063
:1051F800604B9001BDE07045C2057F3F12DBD0C215
:10520800057F0312DC10E4900120F090018FF090EC
:1052180001C7F090019BF09001C6F090013CF07F2F
:105228000512DF277F0412DF277F0312DF277F02A3
:1052380012DF277F0112DF27E4FF12DF277F071223
:10524800C92FEF640160337F0712C92FEF64026032
:10525800299001BDE070239001C4E04402F07DFF75
:105268007F0712DAECE4900183F090013BF09001A3
:0B52780075F0900176F0FF12D3542275
:10CC0100A204E4335401FF90028AE054FE4FFFF086
:10CC1100A205E4335401FE25E0FEEF54FD4EFFF082
:10CC2100A206E4335401FE25E025E0FEEF54FB4E5D
:10CC3100FFF0A207E4335401FE33333354F8FEEF1F
:10CC410054F74EFFF0A208E4335401FEC454F0FE41
:10CC5100EF54EF4EF0900008E0900289F0A209E451
:10CC6100335401FFC43354E0FFA3E054DF4FFFF01E
:10CC7100A20AE4335401FEC4333354C0FEEF54BF5F
:03CC81004EF02250
:10DCCA00EF5407FF900289F0A204E4335401FFC421
:0BDCDA003354E0FFA3E054DF4FF022C2
:10C6CA00200404C2968002D296C291D291C2959059
:10C6DA00028AE0FF139292C291D291EFC31313928E
:10C6EA0092C291D291E01313543F139292C291D203
:10C6FA0091EF131313541F139292C291D291E0C473
:10C70A00540F139292C291D291900289E0FE20E2D4
:10C71A0004C2928002D292C291D291EE20E104C266
:10C72A00928002D292C291D291900289E020E004D2
:10C73A00C2928002D292C291D291EFC413540713CB
:10C74A009292C291D291EFC413135403139292C2DC
:10C75A0091D291C291D291C291D291C291D295D2E3
:02C76A00962215
:10D6D800C2AFE4FDFC200404C2968002D296D29424
:10D6E800C291D291E4FBFAC291ED25E0FDEC33FC46
:10D6F8003093050DBD00010CD2910BBB00010AEB64
:10D70800640A4A70E2C291D291C291D291C291C286
:09D7180094D296D2AFAE04AF0525
:01D7210022E5
:05000E00C290D2902217
:10CF5A00E4FFEF75F003A424CAF582E43401F583F3
:10CF6A00E4F0EF75F003A424CCF582E43401F583F0
:10CF7A00E4F0EF75F003A424CBF582E43401F583E1
:10CF8A00E4F00FEFB408CBE4FFEF75F003A424E25A
:10CF9A00F582E43401F583E4F0EF75F003A424E4A8
:10CFAA00F582E43401F583E4F0EF75F003A424E399
:0ECFBA00F582E43401F583E4F00FEFB410CB00
:01CFC8002246
:10A1050012DE08900008EFF012DE1D90000AEFF055
:10A1150012DE32900009EFF0E4FDED75F003A424A2
:10A12500CCF582E43401F583E4F0900008E0FF30DB
:10A13500E073ED75F003A424CBF582E43401F583D7
:10A14500E0602BED75F003A424CAF582E43401F533
:10A1550083E0FED394054016EE94695011ED75F039
:10A1650003A424CAF582E43401F583E004F0ED7517
:10A17500F003A424CAF582E43401F583E0D3940501
:10A185005058ED75F003A424CAF582E43401F58333
:10A19500E004F0ED75F003A424CCF582E43401F578
:10A1A50083E4F08035ED75F003A424CAF582E43428
:10A1B50001F583E0C394054011ED75F003A424CCAB
:10A1C500F582E43401F58374FFF0ED75F003A42402
:10A1D500CAF582E43401F583E4F0EFC31390000877
:10A1E500F00DED6408600302A11FE4FDED75F003B9
:10A1F500A424E4F582E43401F583E4F090000AE058
:10A2050030E073ED75F003A424E3F582E43401F541
:10A2150083E0602BED75F003A424E2F582E43401BC
:10A22500F583E0FFD394024016EF94665011ED7567
:10A23500F003A424E2F582E43401F583E004F0EDB3
:10A2450075F003A424E2F582E43401F583E0D394A8
:10A25500025058ED75F003A424E2F582E43401F5CB
:10A2650083E004F0ED75F003A424E4F582E4340101
:10A27500F583E4F08035ED75F003A424E2F582E47E
:10A285003401F583E0C394024011ED75F003A42475
:10A29500E4F582E43401F58374FFF0ED75F003A471
:10A2A50024E2F582E43401F583E4F0900009E0A2AC
:10A2B500E713F0A3E013F00DED6410600302A1F1C4
:01A2C5002276
:10DA9000E4FFFEEF7011EE75F003A424CAF582E4F2
:10DAA0003401F583E060047D0180027D00AF050E46
:0FDAB000EEB408DFEF60047E0080027EFFAF0659
:01DABF002244
:10C89C00AE07EE75F003A424CCF582E43401F583E5
:10C8AC00E0B4FF037F0422EE75F003A424CAF582E2
:10C8BC00E43401F583E0FDB405037F0122EDD3944C
:10C8CC0005405DEE75F003A424CBF582E43401F54C
:10C8DC0083E070037F0222EE75F003A424CAF58274
:10C8EC00E43401F583E0FFD3945F500EEF24FB7525
:10C8FC00F01E84E5F070297F0122EE75F003A4246C
:10C90C00CAF582E43401F583E0B46914EE75F003E2
:10C91C00A424CAF582E43401F583745FF07F01220C
:03C92C007F002267
:10C92F00AE07EE75F003A424E4F582E43401F58339
:10C93F00E0B4FF037F0422EE75F003A424E2F58236
:10C94F00E43401F583E0FDB402037F0122EDD394BB
:10C95F0002405DEE75F003A424E3F582E43401F5A3
:10C96F0083E070037F0222EE75F003A424E2F582C8
:10C97F00E43401F583E0FFD3945C500EEF24FE7591
:10C98F00F01E84E5F070297F0122EE75F003A424D8
:10C99F00E2F582E43401F583E0B46614EE75F0033A
:10C9AF00A424E2F582E43401F583745CF07F012264
:03C9BF007F0022D4
:10DEBF00EF75F003A424CBF582E43401F58374FFEE
:02DECF00F0223F
:10DF0500EF75F003A424CBF582E43401F583E4F046
:01DF150022E9
:1095480020005349443A00434D0022004C4F572015
:1095580053504545440048494748205350454544E1
:1095680000554E4445525441424C450054484F52D0
:109578004158004C4F434B45440044455420414E0C
:10958800473A004F42535452554354494F4E0020D6
:1095980000310032003300340035003600253464D1
:1095A800200025342E31660025346400FF9548FFDD
:1095B800954AFF954FFF9552FF9554FF955EFF958D
:1095C80069FF9574FF957BFF9582FF958BFF9597B3
:1095D8000000000000000020202020200020505023
:1095E80050000000005050F850F850502078A070FB
:1095F80028F020C0C810204098186090A040A8907B
:1096080068602040000000001020404040201040CA
:109618002010101020400020A870A8200000202052
:10962800F8202000000000006020400000007800C2
:10963800000000000000006060000810204080006A
:10964800708898A8C88870206020202020707088B2
:1096580010204080F8F810201008887010305090C2
:10966800F81010F880F008088870304080F088887A
:1096780070F80810204040407088887088887070A2
:109688008888780810600040400040400000606012
:1096980000204000102040804020100000F800F812
:1096A8000000804020102040807088081020002092
:1096B8007088B8A8B8807070888888F88888F0881A
:1096C80088F08888F070888080808870E09088882A
:1096D8008890E0F88080F08080F8F88080F08080C2
:1096E80080708880B8888878888888F888888870A2
:1096F800202020202070381010101090608890A032
:10970800C0A09088808080808080F888D8A8A888A9
:1097180088888888C8A89888887088888888887081
:10972800F08888F080808070888888A89068F088A1
:1097380088F0A0908870888070088870F8202020B1
:109748002020208888888888887088888888885019
:1097580020888888A8A8A850888850205088888899
:10976800888850202020F80810204080F870507019
:0497780000000000ED
:10997F00900266E06003029B70900265E060030254
:10998F009B70900267E06003029B70900263E0603F
:10999F0003029B70900262E06003029B7090026969
:1099AF00E06003029B7090026C7407F0A374D1F017
:1099BF00FF7E0712DA5F90026CE0FFA3E0900105D3
:1099CF00CFF0A3EFF07BFF7A95799912C3669002DF
:1099DF006BE075F009A4FF5407600AEF13131354DB
:1099EF001F04FF800F90026BE075F009A4FF1313A3
:1099FF0013541FFF7E007C027D80122D7490010690
:109A0F00E02FFF900105E03EFE90026CF0A3EFF017
:109A1F0012DA5F7BFF7A95799B12C36690026BE037
:109A2F0075F009A4FF5407600AEF131313541F04B2
:109A3F00FF800F90026BE075F009A4FF131313540E
:109A4F001FFF7E007C057D00122D74900106E02F14
:109A5F00FF900105E03EFE90026CF0A3EFF012DAEA
:109A6F005F7BFF7A95799D12C36690026BE075F06C
:109A7F0006A4FF5407600AEF131313541F04FF804B
:109A8F000F90026BE075F006A4FF131313541FFF22
:109A9F00EF75F00CA4FF900106E02FFF900105E099
:109AAF0035F0FE90026CF0A3EFF012DA5F90026CCB
:109ABF00E0FFA3E0900107CFF0A3EFF07BFF7A95D3
:109ACF00799F12C36690026BE075F009A4FF5407EB
:109ADF00600AEF131313541F04FF800F90026BE003
:109AEF0075F009A4FF131313541FFF7E007C027D32
:109AFF0080122D74900108E02FFF900107E03EFEC9
:109B0F0090026CF0A3EFF012DA5F7BFF7A9579A1E8
:109B1F0012C36690026BE075F009A4FF5407600A48
:109B2F00EF131313541F04FF800F90026BE075F0B7
:109B3F0009A4FF131313541FFF7E007C057D001231
:109B4F002D74900108E02FFF900107E03EFE900278
:109B5F006CF0A3EFF012DA5F7BFF7A9579A312C353
:019B6F00668F
:019B700022D2
:08B8730090000AEEF0A3EFF0D3
:10B87B00E4900034F0900266E0600302B985A3E027
:10B88B00FF90000AE0FCA3E0FD6F7001EC70030277
:10B89B00B985900142E07002A3E070589000EB7400
:10B8AB00FFF0A37495F0A374A5F0A3ECF0A3EDF057
:10B8BB007B017A00790C126C1390026BE075F00629
:10B8CB00A4FF5407600AEF131313541F04FF800FD8
:10B8DB0090026BE075F006A4FF131313541FFFEFD8
:10B8EB0075F005A4900034F090026C7407F0A3740B
:10B8FB00DFF0806A90000AE0FCA3E0FDEC1229184F
:10B90B00E4FBFA792078401228769000EB74FFF074
:10B91B00A37495F0A374AAF0A3122FE27B017A0013
:10B92B00790C126C1390026BE075F006A4FF5407B0
:10B93B00600AEF131313541F04FF800F90026BE088
:10B94B0075F006A4FF131313541FFFEF75F005A436
:10B95B00900034F090026C7407F0A374E4F0900242
:10B96B006CE0FEA3E0FF12DA5F7B017A00790C1228
:0AB97B00C36690000BE0900267F035
:01B98500229F
:05B64200900005EFF08F
:10B64700E4A3F0A3F0A3F0A3F0900266E060030286
:10B65700B75B900005E0FF900265E06F700302B7EB
:10B667005B12DBAD900005E075F003A424B4F5820E
:10B67700E43495F583E493FB740193FA740293F928
:10B6870012DE47C374229FFFE49EFE90026BE075B3
:10B69700F006A4FD5407600AED131313541F04FDAD
:10B6A700800F90026BE075F006A4FD131313541F6F
:10B6B700FD7C00122D747D02122D86900006EEF09F
:10B6C700A3EFF024D0FFEE3407FE90026CF0A3EF57
:10B6D700F012DA5F900005E075F003A424B4F58258
:10B6E700E43495F583E493FB740193FA740293F9B8
:10B6F70012C366900142E07002A3E0702390026CCF
:10B707007407F0A374EEF0FF7E0712DA5F9095BA24
:10B71700E493FB740193FA740293F912C3668021D0
:10B7270090026C7407F0A374F1F0FF7E0712DA5FE2
:10B737009095BDE493FB740193FA740293F912C3D5
:10B7470066900005E0900265F0900173E0FEA3E0CB
:04B75700FF12B873B2
:01B75B0022CB
:10DBAD00900265E0601C90026C7407F0A374D0F0D5
:10DBBD00FF7E0712DA5FE4900267F0900265F012C3
:03DBCD00CEE6227F
:08C8050090000AEEF0A3EFF031
:10C80D00E4900034F0900266E0600302C89B900251
:10C81D0064E0FF90000AE0FCA3E0FD6F7001EC60A6
:10C82D006D9000EB74FFF0A37495F0A374B0F0A3BA
:10C83D00ECF0A3EDF07B017A00790C126C139002F1
:10C84D006BE075F006A4FF5407600AEF1313135441
:10C85D001F04FF800F90026BE075F006A4FF131309
:10C86D0013541FFFEF75F005A4900034F090026C87
:10C87D007411F0A37449F0FF7E1112DA5F7B017A17
:0EC88D0000790C12C36690000BE0900264F07C
:01C89B00227A
:05BEC600900005EFF003
:10BECB00E4A3F0A3F0A3F0A3F0900266E0600302FA
:10BEDB00BF96900005E0FF900269E06F700302BF10
:10BEEB009612DB88900005E075F003A424B4F5826C
:10BEFB00E43495F583E493FB740193FA740293F99C
:10BF0B0012DE47C374249FFFE49EFE90026BE07524
:10BF1B00F006A4FD5407600AED131313541F04FD20
:10BF2B00800F90026BE075F006A4FD131313541FE2
:10BF3B00FD7C00122D747D02122D86900006EEF012
:10BF4B00A3EFF02431FFEE3411FE90026CF0A3EF5F
:10BF5B00F012DA5F900005E075F003A424B4F582CB
:10BF6B00E43495F583E493FB740193FA740293F92B
:10BF7B0012C366900005E0900269F0900121E0FE8B
:0BBF8B00A3E0FF12C8057F5B129D625F
:01BF96002288
:10DB8800900269E0601E90026C7411F0A37430F08A
:10DB9800FF7E1112DA5F90026474FFF0E49002696C
:05DBA800F012CEE622A0
:05C1F200900030EFF0A9
:10C1F700E4A3F0A3F0900266E0600302C2AB9000F4
:10C2070030E0FF900263E06F700302C2AB12DC4FB5
:10C21700900030E075F003A424B4F582E43495F57A
:10C2270083E493FB740193FA740293F912DE479047
:10C23700026BE075F006A4FD5407600AED131313B3
:10C24700541F04FD800F90026BE075F006A4FD13E8
:10C257001313541FFD7C00122D74C374289FFFE431
:10C267009EFE7D02122D86900031EFF02490FFE4B0
:10C27700341AFE90026CF0A3EFF012DA5F900030F0
:10C28700E075F003A424B4F582E43495F583E493D0
:10C29700FB740193FA740293F912C366900030E0BD
:04C2A700900263F0AE
:01C2AB002270
:10DC4F00900263E0601890026C741AF0A37490F065
:0FDC5F00FF7E1A12DA5FE4900263F012CEE62223
:05C2AC00900030EFF0EE
:10C2B100E4A3F0A3F0900266E0600302C36590007E
:10C2C10030E0FF900262E06F700302C36512DC6E22
:10C2D100900030E075F003A424B4F582E43495F5C0
:10C2E10083E493FB740193FA740293F912DE47908D
:10C2F100026BE075F006A4FD5407600AED131313F9
:10C30100541F04FD800F90026BE075F006A4FD132D
